:100000000268E232000000000000000265570000B4
:100010000000000265040000000000320000000043
:100020000000000231B40000000000026661000020
:100030000000000264510000000000000000000009
:1000400012004712004722C28E53890F4389107550
:100050008BEB758DCBC28FD28E308FFDC28E22C2BC
:100060008E53890F438910E58AC4242BF58B758D37
:10007000EBC28FD28E308FFDC28E2275F006120138
:100080003C22D20612007BC2062212008212007BA2
:1000900012008212007B12008212007B1200821278
:1000A000007B12008275F01812013C22755707126E
:1000B00030A980E27557061230A980E075F046122B
:1000C000013C22D2061200BC1200BCC206227557A7
:1000D000041230A9D2061237901200BC12379012C7
:1000E00000BC1237901200BC1237901200BC1237BD
:1000F000901200BC1237901200BC123790C2062238
:100100007557051230A91200C375F01812013C1280
:1001100000C3227557031230A912008A12008A22E6
:10012000C205C24012008275F01212013CD205C213
:10013000402212008275F01212013C22120040206F
:100140000907C0F0122E1FD0F0D5F0F0227E007FFC
:100150007090000075F000E49325F0F5F0A3C3E57E
:10016000829EE5839F40F0E5F0700122E5F0C2AD8C
:10017000C2ACD209D203C23ED204C241C205C240BF
:10018000D202C23F7554FA75F0C8120040D5F0FA99
:10019000C203C23ED204C241D205C240D202C23F13
:1001A0007554FA80CF7401126BB440347404126B2E
:1001B000B4402D7404126B6F7401126B6FC2AF7573
:1001C00018C075190B7400543F4440F51A1203EE21
:1001D000C2AF7518C0751900751A681203EED322E4
:1001E000C3227404126BB4401A7404126B6FC2AF52
:1001F0007518C075190B7400543F4440F51A12036A
:10020000EED322C322C5342534C53422E55324EE6F
:100210004008D203C23ED204C2413098EFC298E5F2
:1002200099120205223099FDC299F5991202052210
:10023000785A7400F2087401F2087401F20874002C
:10024000F2087400F2087400F2087406F222785F73
:10025000E2C0E0785A797375F007E2F70809D5F043
:10026000F9785FE2D0F0B5F0E82274A0120334E52B
:100270002F120361E8120361E71203610908D53008
:100280000412039522E87004052F8004541F70E8BF
:1002900012039512004774A0120334E52F12036174
:1002A000E812036180D274A0120334E52F120361B7
:1002B000E8120361E31203610908D53004120395C3
:1002C00022E87004052F8004541F70E81203951271
:1002D000004774A0120334E52F120361E812036192
:1002E00080D274A0120334E52F120361E812036177
:1002F00074A112033412037FF709D5300412039559
:1003000022C281D2800000C28080EA74A01203342D
:10031000E52F120361E812036174A1120334120382
:100320007FF309D5300412039522C281D2800000E8
:10033000C28080EA7A08D281D2800000000000C228
:10034000810000C280335005D28102034FC281D2A6
:10035000800000C280DAEED28100D2800000C2802C
:10036000227A08335005D28102036DC281D2800007
:1003700000C280DAEED28100D2800000C280227AF0
:1003800008D281C280000000D280C3308101B33323
:10039000DAF1C28022C2810000D2800000D2812224
:1003A00074A0120334E52F120361E8120361E9120D
:1003B0000361D530F91203952274A0120334E5834A
:1003C000120361E58212036174A1120334790012F1
:1003D000037F29F9A3E5836B700AE5826C7005122F
:1003E0000395E922C281D2800000C28080E1535986
:1003F0000F53580F5318F053190FC2AFE558232469
:100400002AF8E5184519F208E51AF2055853580F6D
:10041000E558B55905055953590FD2AF22E559B5DD
:100420005805740078002223242AF8E2C0E008E28C
:10043000F8D0E022302CFDD20675F00612013CC245
:100440000675F01412013CE53CC22C2230611720E5
:100450002C1475A0FFC0E0E8C0E0C0D0020467D053
:10046000D0D0E0F8D0E02275A0EF0000000000003E
:10047000E5A075A0DF30E03A30E14730E25430E3E8
:100480005DE5A075A0BF30E02D30E13A30E22030CC
:10049000E350E5A075A07F30E02030E12D30E2365A
:1004A000E5A030E01930E12630E22F74FF8037E418
:1004B0008034740180307402802C740380287404AA
:1004C0008024740580207406801C740780187408CA
:1004D000801474098010740A800C740B800874BC3A
:1004E000800474BD8000B53A0EE53B600FD53B0C2F
:1004F000E53AB4FF0D8005F53A753B0175A00F0292
:10050000045FD22CF53C80F42285832FA88279FFEA
:100510007530201203A0120047E5822420F5825096
:10052000020583229000007FC0120509120509DF31
:10053000F8229031007F08120509DFFB222222C237
:1005400044C245D227D226755E03122F1222797338
:10055000770509774709770B0977C0097704097789
:1005600001752F307800797375300612026A120017
:100570004722752F30780079737530061202E279C0
:1005800075E7640B227973E4A20C92E0A20D92E16C
:10059000A20E92E2A20F92E3A21092E4A21192E5BF
:1005A000A21292E6A21392E7F709E4A21492E5A23E
:1005B0001592E6F7752F2A78A0797375300212022A
:1005C0006A12004722752F2A78A0797375300212BB
:1005D00002E27973E7A2E0920CA2E1920DA2E2920C
:1005E0000EA2E3920FA2E49210A2E59211A2E6926B
:1005F00012A2E7921309E7A2E59214A2E69215224D
:10060000E4A22192E2A25992E3A25D92E4A2239293
:10061000E67973F7E4A22292E0A20892E1A2569250
:10062000E2A25792E3A27192E4A25492E6A25192FE
:10063000E709F7E4A24F92E0A25092E1A25C92E3B4
:10064000A25A92E4A25B92E509F7E4A26092E0A2CA
:100650006192E1A25E92E2A25F92E3A26292E4A2C0
:100660006392E5A26492E6A26592E709F7E409F7CE
:10067000E409F7E409F7E409F7752F2A784079735C
:1006800075300812026A12004722752F2A784079C5
:10069000737530081202E27973E7A2E29221A2E3B5
:1006A0009259A2E4925DA2E6922309E7A2E0922287
:1006B000A2E19208A2E29256A2E39257A2E49271BA
:1006C000A2E69254A2E7925109E7A2E0924FA2E17A
:1006D0009250A2E3925CA2E4925AA2E5925B09E7EF
:1006E000A2E09260A2E19261A2E2925EA2E3925F36
:1006F000A2E49262A2E59263A2E69264A2E7926506
:1007000022C2E0A22492E092E192E2A22592E49237
:10071000E592E67973F7752F2A782279737530019F
:1007200012026A12004722752F2A782279737530D7
:10073000011202E27973E7A2E09224A2E492252258
:10074000752F2A7820793575300112026A12004718
:1007500022752F2A782079357530011202E2227530
:100760002F2A7821793675300112026A1200472249
:10077000752F2A782179367530011202E222752F01
:100780002A7860796E7530011202A6120047752F23
:100790002A7861796F7530011202A6120047752F11
:1007A0002A786279707530011202A6120047752FFF
:1007B0002A786379717530011202A6120047752FED
:1007C0002A786479727530011202A6120047752FDB
:1007D0002A786579737530011202A6120047752FC9
:1007E0002A786679747530011202A6120047752FB7
:1007F0002A786779757530011202A6120047752FA5
:100800002A786D79767530011202A6120047752F8D
:100810002A786E79777530011202A6120047227588
:100820002F2A7860796E75300112030B752F2A78A4
:1008300061796F75300112030B752F2A7862797018
:1008400075300112030B752F2A78637971753001A9
:1008500012030B752F2A7864797275300112030B1D
:10086000752F2A7865797375300112030B752F2A5D
:100870007866797475300112030B752F2A786779C1
:100880007575300112030B752F2A786D79767530E6
:100890000112030B752F2A786E79777530011203D8
:1008A0000B22752F2A788079787530011202A612F2
:1008B0000047752F2A788179797530011202A612C6
:1008C0000047752F2A7882797A7530011202A612B4
:1008D0000047752F2A7883797B7530011202A612A2
:1008E0000047752F2A7884797C7530011202A61290
:1008F0000047752F2A788D797D7530011202A61276
:100900000047752F2A788E797E7530011202A61263
:10091000004722752F2A7880797875300112030BF1
:10092000752F2A7881797975300112030B752F2A7A
:100930007882797A75300112030B752F2A788379C2
:100940007B75300112030B752F2A7884797C753002
:100950000112030B752F2A788D797D7530011203F2
:100960000B752F2A788E797E75300112030B227554
:100970002F2A782F79717530011202E2752F2A78AB
:100980003079727530011202E2E572F4F5FD2275DC
:100990002F2A782F797175300112026A120047757B
:1009A0002F2A7830797275300112026A120047E5F9
:1009B00072F4F5FD22752F2A78E0797375300912EB
:1009C00002E27873790075F009E6F30809D5F0F9C9
:1009D000227873790075F009E3F60809D5F0F97506
:1009E0002F2A78E0797375300912026A12004722C3
:1009F00078657973E2F70809E2F7752F2A78237989
:100A00007375300212026A12004778677973E2F751
:100A10000809E2F7752F2A782579737530021202DA
:100A20006A12004722752F2A7823797375300212D3
:100A300002E278737965E6F30809E6F3752F2A7800
:100A40002579737530021202E278737967E6F3084C
:100A500009E6F322752F247880791E753002120280
:100A60006A12004722752F247880791E7530021291
:100A700002E222788879777A28E56C75F00484FAA6
:100A8000C0F080021819E7F5F066540F7035DA0CE3
:100A9000D0E0602DFA18E7C4F5F0801618E7C4F529
:100AA000F066540F701DDADCD0E06015FA1819E713
:100AB000F5F0E4D333DAFCFAE65AC5F05A65F07083
:100AC00004E422D0E0740122C2327878798B7A066D
:100AD000E7540FF7EA30E004E6088002E6C4540F5A
:100AE000B40F0AB70F0A20321BE4C23222B70F0339
:100AF0007401222032FAF5F0893E676002D2320991
:100B0000DACE80E2E5F0A93EC3975002F404146007
:100B100003B408DCE4D23222120AC8701C30321945
:100B2000202217D2317405126B6FC2AF7518508531
:100B3000831985821A1203EEE4220422752F247889
:100B40008A79737530051202E2120A7322752F2416
:100B5000788A797375300512026A12004722752F60
:100B600024788279737530081202E2120A732275B2
:100B70002F24788279737530081202E2120B182242
:100B8000752F247882797375300512026A12004736
:100B900022752F247887797875300312026A120043
:100BA00047227537FEE58245836021C082C083E518
:100BB0008224A0F582E5833424F58385832FA882DF
:100BC00079377530011202E2D083D08222C082C010
:100BD00083E58224A0F582E5833424F58385832F81
:100BE000A882793775300112026A120047D083D08B
:100BF0008222C082C083E5822460F582E58334F0DE
:100C0000F5835008120C8CD083D08222D083D082FE
:100C1000C082C083125C37D083D082120BA2C08204
:100C2000C083120CE785832FA88279737530081270
:100C300002E2D083D082227004A227804E20680C6A
:100C40002400F58274243400F583800A2480F58220
:100C500074233400F58385832FA88279737530015E
:100C60001202E27873E6B40103D3801FB40203C317
:100C7000801920E716C0E0030303540F244AF8D07C
:100C8000E0540704F5F0E213D5F0FC22C082C083E3
:100C9000E5822460F582E5833431F58385832FA8CE
:100CA0008279387530011202E2D083D082C082C0CE
:100CB00083E5822480F582E5833431F58385832FB3
:100CC000A88279377530011202E2D083D082C082C7
:100CD000C083120D1F85832FA88279737530081287
:100CE00002E2D083D08222E58275F008A42420F5A8
:100CF00082500205F0C0F0E58375F008A4D0F0251D
:100D0000F02400F58322C082C083120CE785832F74
:100D1000A882797F7530081202E2D083D08222E562
:100D20008275F008A42420F582500205F0C0F0E599
:100D30008375F008A4D0F025F02431F58322C08219
:100D4000C083E5822460F582E58334F0F583120DDB
:100D50001F85832FA882797F7530081202E2D08325
:100D6000D08222C082C083E5822460F582E583348C
:100D7000F0F583120D1F85832FA8827973753008D3
:100D80001202E2D083D08222787F790A74FF56085B
:100D9000D9FC046028751B20751C31900FA0756567
:100DA000A875660F120DC56017751B20751C009085
:100DB00000007565E8756603120DC56003740122B5
:100DC000120BF2E422851C2FA81B797375300512D3
:100DD00002E2120A736017E51B2408F51B50020596
:100DE0001CA3E583B566DEE582B565D9740122757D
:100DF0001B25751C31900FA07565A875660F120E26
:100E00001F6017751B25751C009000007565E8753F
:100E10006603120E1F6003740122120BF2E4228596
:100E20001C2FA81B79787530031202E2120B186090
:100E300017E51B2408F51B5002051CA3E583B566C6
:100E4000DEE582B565D974012230390DE533B4434E
:100E500008E53124FE500280F0787F7A0579A8E613
:100E6000540FC4F5F008E6540F45F0F70809DAEF1F
:100E7000227F14C283120040308717D283120040B1
:100E800020870FDFEEC2837554FA75A61E75A6E1A2
:100E9000D322C283C3227F14C28312004030B21710
:100EA000D28312004020B20FDFEEC2837554FA7570
:100EB000A61E75A6E1D322C283C322D282D2B67FF8
:100EC00028C28312004730B617D28312004720B6DB
:100ED0000FDFEEC2837554FA75A61E75A6E1D32204
:100EE000C283C322C203C23EC204C241C205C24081
:100EF000120EBBC201400C120E96D2014005020F29
:100F000042D206C203C23EC204C241C205C24075FB
:100F1000F005120040D5F0FA75A61E75A6E1120E76
:100F2000BB40DE120E9640D9020F2BC2061210AF44
:100F300075F005120040D5F0FA75A61E75A6E102FF
:100F400068B3C206120FCB40141205726003121070
:100F5000EC120FBB400712103B12127F2278B5E251
:100F60004402F27406126B6F12153840031212938A
:100F7000D203C23ED204C241C205C240D202C23F25
:100F8000C2097554FA75F0C8120040D5F0FAD206BD
:100F900075F064120040D5F0FA120E96401A120E47
:100FA000BB401575F064120040D5F0FAC206120E6F
:100FB000964005120EBB50B8020F039000007B3024
:100FC0007C001203B97002C322D32212081F120937
:100FD00013786EE2B4FF62786FE2B4FF5C7870E27F
:100FE000B4FF567871E2B4FF507872E2B4FF4A78E9
:100FF00073E2B4FF447874E2B4FF3E7875E2B4FF64
:10100000387876E2B4FF327877E2B4FF2C7878E271
:10101000B4FF267879E2B4FF20787AE2B4FF1A7838
:101020007BE2B4FF14787CE2B4FF0E787DE2B4FF7B
:1010300008787EE2B4FF02D322C3221205C575A64A
:101040001E75A6E112068A75A61E75A6E11207276F
:1010500075A61E75A6E112075175A61E75A6E112AA
:10106000077075A61E75A6E112081F75A61E75A647
:10107000E112091375A61E75A6E1120A6575A61E72
:1010800075A6E11209B575A61E75A6E1120A2575A9
:10109000A61E75A6E1752F247800796F75300112B0
:1010A00002E275A61E75A6E112096F12153822120A
:1010B0001125125D4F9000007537FE125BEF120B89
:1010C00080120B911200B4200105125A9180031274
:1010D0005B4A125CD212053212053D1239A7227802
:1010E0007F79737A08E6F70809DAFA22900000128D
:1010F0000D06C01EC01F121125D01FD01E1215389C
:10110000120A541210DF9000007538007537FE1275
:101110005BEF120B80120B91125CD212053212059A
:101120003D1239A722120524751E30751F30121585
:1011300038D20CC20DC20EC20FC210C211C212C2EE
:1011400013C214C215C221C222C223C251C254C248
:101150004FC25AC25BC25CC259C25DD260D261C288
:101160005EC25FD266D267C208C271D256D25778C9
:10117000657422F2087400F278677406F20874004D
:10118000F2C224C225753504753609786E7401F2F1
:10119000786F7402F278707404F278717400F278E7
:1011A000727400F278737400F278747400F27875D7
:1011B0007400F278767400F278777400F2787874BC
:1011C00063F2787DF278797407F2787EF2787A7437
:1011D00000F2787B7400F2787C7400F2787D740001
:1011E000F2787E7400F2756F02752F247800796FA3
:1011F00075300112026A120047126B19120A54125A
:10120000058512060012070112074012075F120738
:101210007E1208A21209D112054E125F8E1209F039
:10122000787376FF752F307810797375300112025C
:101230006A12004722752F327800797375300412D4
:1012400002E2E5732574246AB5750BE57365746471
:1012500050B57602C322D322851E73851F74E573B1
:101260002574246AF575E57365746450F576752FF9
:10127000327800797375300412026A120047221224
:101280001235400BE51EB57306E51FB57401221239
:10129000125822121235400685731E85741F22755E
:1012A0002F237862797375300A1202E2787F79739E
:1012B00075F00AE7B4FF02802CB43C240809D5F08D
:1012C000F2900FE8752F237860793875300112029B
:1012D000E2752F23786179377530011202E2E4223A
:1012E00066540F60D7740122E582B4E807E583B441
:1012F0000F02D322C322752F237862797375300AC7
:1013000012026A120047753800752F237860793809
:1013100075300112026A120047752F237861793700
:1013200075300112026A120047221213BA402FE5EB
:101330008275F006A4F582A8F0E58375F006A4286E
:10134000F583E5822400F582E5833450F583C0827D
:10135000C08379AD7406126A50D083D08222E582B0
:1013600075F006A4F582A8F0E58375F006A428F5CB
:1013700083E58224E0F582E58334D3F58385832FEA
:10138000A88279AD7530061202E2227874E6540F15
:101390002323F67875E6541F030303F5F05403780E
:1013A0007446F67876E6541FC5F054E045F078753B
:1013B000F622C3EC9FEB9EEA9D22C082C083E582A9
:1013C0002460E58334F05010E5822458E58334F03E
:1013D0004006D083D082D322D083D082C322E5833B
:1013E000B40F08E582B4E80302143712132A78AD6B
:1013F000E6B4FF0302143712024E12138B7873E621
:10140000FA08E6543FFB08E6FC78ADE6FD08E65432
:101410003FFE08E6FF1213B2401F7873E6FA08E6B3
:10142000543FFB08E6FC78B0E6FD08E6543FFE08B2
:10143000E6FF1213B25002C322D3227809E2B408A5
:101440000050F6C0E0F582758300120D1F85832FD2
:10145000A882790A7530081202A6120047D0E0C0AF
:10146000E07583312460F5825002058385832FA8BF
:101470008279127530011202A6120047D0E0C0E056
:101480007583312480F5825002058385832FA882DD
:1014900079137530011202A6120047D0E075F006EC
:1014A000A424A0F582E5F03431F58385832FA8824A
:1014B00079147530061202A612004712053DC322A8
:1014C0007809E2B4080050F7C0E0F5827583001295
:1014D0000D1F85832FA882790A75300812030BD05F
:1014E000E0C0E07583312460F58250020583858376
:1014F0002FA882791275300112030BD0E0C0E0757D
:1015000083312480F5825002058385832FA8827958
:101510001375300112030BD0E075F006A424A0F57A
:1015200082E5F03431F58385832FA88279147530F4
:101530000612030BC3741122C082C083906FB2E401
:1015400093B430004026B43A005021F5F0A3E49360
:10155000B430004017B43A00501285F01EF51F90C9
:1015600000B5E04401F0D083D082D3229000B5E0F2
:1015700054FEF0D083D082C3220022D2B512157956
:10158000C2B512157922C2B5C284121579D2B5122C
:101590001579D284121579C2B512157975F0083310
:1015A000928412157BD5F0F722D2B775F008D2B528
:1015B000121579A2B7C2B512157933D5F0F022C24F
:1015C000B5C284121579D2B5121579D28412157963
:1015D000C2B5121579D28412157B12157B12157BB8
:1015E00022D2B5D2B77473121586744B1215867455
:1015F0005012158612005F74081215861215A92361
:10160000243F543F4480121586746B1215861200D5
:1016100047746812158612005F74601215861215E1
:10162000BF22C2ABC28ED2AF75F00AC0F0745512A1
:101630001586D2B5D2B775F01ED5F0FDD0F0D5F035
:10164000EA22200A16200B1330430E755700123081
:10165000A975570012319BC243C32230B6EA300A43
:10166000067557001230A9300B0675570012319BD2
:10167000C243D322D23CD243742002168CD23C8087
:1016800002C23CD2437440300902740CF5517554C7
:10169000FA121836753900C23BC23AC22C753CFFAB
:1016A000C253E5516027121642205321203A1E20D2
:1016B0003B1B302C30203C1575516012043412183D
:1016C00043400AB40B11D23B206802D269C28EC2D9
:1016D000ABD2AF7554FA22533907F8E539248BC8D9
:1016E000F6053980BD75F005120040D5F0FA121AE2
:1016F000FB122E1F75F005120040D5F0FA121AFBEE
:10170000122E1F30610E12171E5009756C28D23A26
:10171000D26980B9808C1217E7121622C3221215E3
:10172000E112182A757010C28E53890F438910E593
:101730007060E3202CE3C28E758B01758D00C28F23
:10174000D28EA2B792363036E6208FCDA2B7303691
:1017500001B350F5758B19758DFCC28F7908308FE8
:10176000FD758B0D758DFEC28FA2B7303601B3406B
:10177000BE208FBBA2B7303601B350F5758B1975FB
:101780008DFCC28FD9D8787F790B7B007A057C00DD
:10179000C234308FFD758B0D758DFEC28FA2B7924E
:1017A00037203601B35002B234EC33FC208F80A2D4
:1017B000B7303701B350F5758B19758DFCC28FDAD0
:1017C000D1D914EC20E00603540F6B600302172FED
:1017D0001216221217F22230340302172FEC035490
:1017E0000FF6086BFB80A578B774FFF278B674002B
:1017F000F22275F00A78B7797F7A00E267701008F4
:1018000009D5F0F778B6E2601ED5E01BF2D322E7E7
:10181000F2540F70010A0809D5F0F478B6EAB4085A
:1018200000740140027403F2C322E4800274FF7862
:101830007F75F00A8007788B75F00674FFF608D57F
:10184000F0FB22107006C322C3D27022206842B47B
:10185000BC24756411752F2A78C079737530011214
:1018600002E2A264926F7873E6C082C083121912FA
:10187000D083D08280D3B4BD16756412752F2A78B8
:10188000C179737530011202E2A265926F80D78030
:10189000B7B4BC16756411752F2A78C47973753086
:1018A000011202E2A262926F80BCB4BD16A26392E2
:1018B0006F756412752F2A78C5797375300112021D
:1018C000E280A3808300010204093D404142434479
:1018D00045464748494A4B4C4E4F50515253F5F0FC
:1018E0009018C5E493B5F002C322A3E583B418F3BE
:1018F000E582B4DEEED322E583B40F0122E582B4A3
:10190000E90122C2AF7518E085831985821A120396
:10191000EE22900FE9306F3FC0E012523B4027E5C6
:1019200064B41111206807E53720E3298018E537F2
:1019300020E1228011206807E53720E4188007E5C0
:101940003720E2118000D0E0123ECE1200CED3222A
:101950001200ACD322D0E0B4FF04D253D322B4019E
:101960000280F7B4000280F4B4020D1218F71231AD
:101970009D121BC450D580D8B404191218F7123127
:101980009DE5642453C2AFF51A7519007518C0128D
:1019900003EE80BCB4092A3027C27408126BB4402D
:1019A000BB1218F712319D7404126B6FC2AF751819
:1019B000C075190BE564543F4440F51A1203EE80DC
:1019C0008FB43C0E1218F712319DE564122FEA0213
:1019D0001950B43D2C20271A121D8B500602194BAA
:1019E00002195C1218F712319D121D42756D4002EA
:1019F00019501218F712319D121D23756D400219EE
:101A000050B440091218F7122E50021950B441096F
:101A10001218F7122E91021950B442091218F71237
:101A20002E78021950B443091218F7122E690219C0
:101A300050B4440B7400126B6F122EAC021950B4E8
:101A4000450B7400126BA0122EBD021950B4461241
:101A50007400126BB440EB7400126B4F122EAC0288
:101A60001950B4470B7402126B6F122ECE0219502C
:101A7000B4480B7402126BA0122EDF021950B44945
:101A8000127402126BB440EB7402126B4F122ECE22
:101A9000021950B44A0B7403126B6F122EF0021924
:101AA00050B44B0B7403126BA0122F01021950B4E7
:101AB0004C127403126BB440EB7403126B4F122E72
:101AC000F0021950B44E093027030219F202195CD2
:101AD000B44F062027F70219D8B450087400122F0B
:101AE0009C021950B45104744080F3B452047480C1
:101AF00080ECB4530474C080E5C322E56070030237
:101B00001B82B40119C2AF75186075190F751AFAE6
:101B10001203EE755E03122F17121B898061B40247
:101B200019122F17C2AF75187075190F751AFA129E
:101B300003EE755E03122F4380DFB40316C2AF7548
:101B4000186075190F751AE01203EE755E03122FF7
:101B50001780C6B40419122F17C2AF751870751903
:101B60000F751AE01203EE755E03122F4380AAB4BC
:101B700005051201E28008B40605121D7B80007580
:101B800060001263271237902230270BC203C23E37
:101B9000D202C23FD24322D203C23EC202C23FD2CD
:101BA0004322E535F555A228B36001D34002C24B6C
:101BB0009228D24AD24322755501C22822305003BE
:101BC000121BB722204517121DC24012121BA2C2BF
:101BD000AF751810E564121BED1203EED322C2AFED
:101BE000751820E564121BED1203EEC322B4000742
:101BF00075190F751AFF22B4010775190F751AE1CF
:101C000022B4020775190F751AE222B40307751979
:101C10000F751AE322B4040775190F751AE422B47C
:101C2000050775190F751AE522B4060775190F75A2
:101C30001AE622B4070775190F751AE722B40807C8
:101C400075190F751AD822B4090775190F751AD9A5
:101C500022B40A0775190F751ADA22B40B07751921
:101C60000F751ADB22B40C0775190F751ADC22B434
:101C70000D0775190F751ADD22B40E0775190F754A
:101C80001ADE22B40F0775190F751ADF22B4110777
:101C900075190F751AD122B4120775190F751AD25A
:101CA00022B4130775190F751AD322B414077519C6
:101CB0000F751AD42275190F751AD422C2AF751870
:101CC000C0751900751A011203EEE55530281D2064
:101CD000443C204F037555022536500274FFF550E1
:101CE000205B03123F35786374FFF222D22E7552C7
:101CF000FFC2AF75185075190F751AFF1203EE3039
:101D0000270C7408126BB440057404126B6F2275B3
:101D10005000C230C2AF7518C0751900751A021292
:101D200003EE22C227122F17755E03C2AF7518602B
:101D3000E564121BED1203EEC22E121B89D24AD2A9
:101D40004322D227122F17C2AF751870E564121BF9
:101D5000ED1203EE122F43755E03121B89D24AD295
:101D6000432212206640121223AF400D1226F84083
:101D700008122A2D4003122D62E42212209212230F
:101D8000DB122724122A59122D8E222027321220EC
:101D90007C402E12208740291223C540241223D0D4
:101DA000401F12270E401A1227194015122A4340CD
:101DB00010122A4E400B122D784006122D8340013E
:101DC000C32212207140121223BA400D1227034081
:101DD00008122A384003122D6D22A286300C01B35E
:101DE000E54733F54722104703022122300907C394
:101DF0007547000220A0E547540760F764076003B9
:101E0000022120786EE2B40302800620200320160F
:101E10002FD216786EE224AC4013E225E0F5F004F0
:101E2000901FBE93C5F093C0F0C0E0E222786EE24E
:101E3000F5F0C2AF75189075190985F01A1203EE06
:101E4000022120121B891200AC0221207401121CF5
:101E5000BC022120756401121BC440E7120100027C
:101E60002120756401D3122FB10221207406126B58
:101E70006F021E2D755D05021E2D1201A502212087
:101E800030270A7408126BB440031201E2022120C9
:101E9000205C03021E2D022120D37401122F4C025C
:101EA0001E2D3027167408126BB4400F7404126B89
:101EB000B44008122F354003021E2D022120740168
:101EC000122FEA021E43202717121D8B5006120103
:101ED00000022120756401756D40121D42021E43EF
:101EE000756401121D23756D40021E437401122E8C
:101EF000500221207401122E910221207401122E11
:101F0000780221207401122E690221207400126BC4
:101F10006F7401122EAC021E437400126BA0740188
:101F2000122EBD021E437400126BB440EC740012FA
:101F30006B4F7401122EAC021E437402126B6F744D
:101F400001122ECE021E437402126BA07401122ED7
:101F5000DF021E437402126BB440EC7402126B4F2A
:101F60007401122ECE021E437403126B6F740112A1
:101F70002EF0021E437403126BA07401122F010293
:101F80001E437403126BB440EC7403126B4F740164
:101F9000122EF0021E43302703021EE002212020F1
:101FA00027FA021EC974004401122F9C021E4374BA
:101FB00040021FA77480021FA774C0021FA71E51F2
:101FC0001E4C1E541E621E2D1E6C1E6C1E741E7A2C
:101FD0001E8021201E2D21201E901E991EA2212030
:101FE00021202120212021202120212021202120E9
:101FF00021202120212021202120212021202120D9
:1020000021202120212021202120212021202120C8
:1020100021202120212021202120212021202120B8
:1020200021202120212021202120212021202120A8
:102030002120212021201EBE1EC6212021201EEC91
:102040001EF41EFC1F041F0C1F191F261F3A1F47DA
:102050001F541F681F751F8221201F961F9F1FA5D9
:102060001FAF1FB41FB9786EE2B40103A21622C3DA
:1020700022786EE2B40B03A21622C322786EE2B479
:102080000D03A21622C322786EE2B40803A2162220
:10209000C322786EE2B40903C21622B409FC80F8A8
:1020A000786EE2B403028009202006201603022184
:1020B00020C216786EE260F6B40109121BBD121D33
:1020C0000F022120B40203022120B40312121D8B3F
:1020D0004009756401C3122FB18045D2168041B406
:1020E0000802803CB409028037B40D05205C3180C1
:1020F0001CB40E08C37401122F4C8011B40F0302DC
:1021000020E724CE5007786EE224AC5013786EE2BC
:10211000F5F0C2AF7518A075190985F01A1203EE13
:10212000D24722A287300D01B3E54833F54822108B
:10213000470302246B300907C37548000223E9E511
:1021400048540760F764076003022469786FE2B4BB
:102150000302800620200320172FD217786FE22475
:10216000AC4013E225E0F5F00490230793C5F0930B
:10217000C0F0C0E0E222786FE2F5F0C2AF751890CF
:1021800075190A85F01A1203EE022469121B8912CE
:1021900000AC0224697402121CBC0224697564023A
:1021A000121BC440E7120100022469756402D312B5
:1021B0002FB10224697406126B6F022176755D05DA
:1021C0000221761201A502246930270A7408126BD5
:1021D000B440031201E2022469205C03022176026A
:1021E0002469D37402122F4C02217630271674080A
:1021F000126BB4400F7404126BB44008122F3540B8
:10220000030221760224697402122FEA02218C2033
:102210002717121D8B5006120100022469756402F3
:10222000756D40121D4202218C756402121D2375CA
:102230006D4002218C7402122E5002246974021225
:102240002E910224697402122E78022469740212FB
:102250002E690224697400126B6F7402122EAC0294
:10226000218C7400126BA07402122EBD02218C749A
:1022700000126BB440EC7400126B4F7402122EAC5F
:1022800002218C7402126B6F7402122ECE02218C0A
:102290007402126BA07402122EDF02218C740212DF
:1022A0006BB440EC7402126B4F7402122ECE0221FA
:1022B0008C7403126B6F7402122EF002218C740363
:1022C000126BA07402122F0102218C7403126BB4E2
:1022D00040EC7403126B4F7402122EF002218C300A
:1022E00027030222290224692027FA0222127400FD
:1022F0004402122F9C02218C74400222F07480024E
:1023000022F074C00222F0219A2195219D21AB2157
:102310007621B521B521BD21C321C92469217624A7
:102320006921D921E221EB246924692469246924E3
:102330006924692469246924692469246924692435
:102340006924692469246924692469246924692425
:102350006924692469246924692469246924692415
:102360006924692469246924692469246924692405
:1023700069246924692469246924692469246922F7
:1023800007220F246924692235223D2245224D224D
:10239000552262226F22832290229D22B122BE22E8
:1023A000CB246922DF22E822EE22F822FD230278E4
:1023B0006FE2B40103A21722C322786FE2B40B03C9
:1023C000A21722C322786FE2B40D03A21722C32200
:1023D000786FE2B40803A21722C322786FE2B4092F
:1023E00003C21722B409FC80F8786FE2B4030280BC
:1023F00009202006201703022469C217786FE260C3
:10240000F6B40109121BBD121D0F022469B40203A8
:10241000022469B40312121D8B4009756402C312B1
:102420002FB18045D2178041B40802803CB4090224
:102430008037B40D05205C31801CB40E08C37402D3
:10244000122F4C8011B40F0302243024CE50077891
:102450006FE224AC5013786FE2F5F0C2AF7518A0AC
:1024600075190A85F01A1203EED24722A2B2300E75
:1024700001B3E54933F549221047030227B4300977
:1024800007C3754900022732E549540760F764071E
:1024900060030227B27870E2B403028006202003B2
:1024A00020182FD2187870E224AC4013E225E0F512
:1024B000F00490265093C5F093C0F0C0E0E222787B
:1024C00070E2F5F0C2AF75189075190C85F01A120C
:1024D00003EE0227B2121B891200AC0227B274036A
:1024E000121CBC0227B2756403121BC440E7120120
:1024F000000227B2756403D3122FB10227B274060B
:10250000126B6F0224BF755D050224BF1201A50284
:1025100027B230270A7408126BB440031201E2029A
:1025200027B2205C030224BF0227B2D37403122F08
:102530004C0224BF3027167408126BB4400F740489
:10254000126BB44008122F3540030224BF0227B299
:102550007403122FEA0224D5202717121D8B500670
:102560001201000227B2756403756D40121D42020C
:1025700024D5756403121D23756D400224D57403A0
:10258000122E500227B27403122E910227B2740346
:10259000122E780227B27403122E690227B2740039
:1025A000126B6F7403122EAC0224D57400126BA050
:1025B0007403122EBD0224D57400126BB440EC7467
:1025C00000126B4F7403122EAC0224D57402126BEE
:1025D0006F7403122ECE0224D57402126BA0740302
:1025E000122EDF0224D57402126BB440EC74021276
:1025F0006B4F7403122ECE0224D57403126B6F74CA
:1026000003122EF00224D57403126BA07403122F50
:10261000010224D57403126BB440EC7403126B4FA7
:102620007403122EF00224D53027030225720227EC
:10263000B22027FA02255B74004403122F9C022467
:10264000D57440022639748002263974C0022639B6
:1026500024E324DE24E624F424BF24FE24FE2506FD
:10266000250C251227B224BF27B22522252B25347D
:1026700027B227B227B227B227B227B227B227B292
:1026800027B227B227B227B227B227B227B227B282
:1026900027B227B227B227B227B227B227B227B272
:1026A00027B227B227B227B227B227B227B227B262
:1026B00027B227B227B227B227B227B227B227B252
:1026C00027B227B227B227B22550255827B227B202
:1026D000257E2586258E2596259E25AB25B825CCDD
:1026E00025D925E625FA2607261427B226282631DD
:1026F000263726412646264B7870E2B40103A218FD
:1027000022C3227870E2B40B03A21822C32278708D
:10271000E2B40D03A21822C3227870E2B40803A227
:102720001822C3227870E2B40903C21822B409FC4B
:1027300080F87870E2B40302800920200620180394
:102740000227B2C2187870E260F6B40109121BBD0C
:10275000121D0F0227B2B402030227B2B4031212F1
:102760001D8B4009756403C3122FB18045D21880B8
:1027700041B40802803CB409028037B40D05205CE6
:1027800031801CB40E08C37403122F4C8011B40F97
:102790000302277924CE50077870E224AC501378D6
:1027A00070E2F5F0C2AF7518A075190C85F01A1219
:1027B00003EED24722104703022AE9300903022A16
:1027C00067301401B34003022A677876E2B403024B
:1027D0008006202003201E2FD21E7876E224AC40F3
:1027E00013E225E0F5F00490298593C5F093C0F03D
:1027F000C0E0E2227876E2F5F0C2AF751890751964
:102800000785F01A1203EE022AE7121B891200ACA8
:10281000022AE7740E121CBC022AE775640E121B12
:10282000C440E7120100022AE775640ED3122FB1EB
:10283000022AE77406126B6F0227F4755D05022702
:10284000F41201A5022AE730270A7408126BB4407B
:10285000031201E2022AE7205C030227F4022AE7BE
:10286000D3740E122F4C0227F43027167408126B03
:10287000B4400F7404126BB44008122F35400302A9
:1028800027F4022AE7740E122FEA02280A202717DB
:10289000121D8B5006120100022AE775640E756D39
:1028A00040121D4202280A75640E121D23756D40E8
:1028B00002280A740E122E50022AE7740E122E916C
:1028C000022AE7740E122E78022AE7740E122E697D
:1028D000022AE77400126B6F740E122EAC02280AE3
:1028E0007400126BA0740E122EBD02280A7400121E
:1028F0006BB440EC7400126B4F740E122EAC0228B5
:102900000A7402126B6F740E122ECE02280A740221
:10291000126BA0740E122EDF02280A7402126BB41E
:1029200040EC7402126B4F740E122ECE02280A7401
:1029300003126B6F740E122EF002280A7403126BCE
:10294000A0740E122F0102280A7403126BB440EC1B
:102950007403126B4F740E122EF002280A302703F4
:102960000228A7022AE72027FA0228907400440EC2
:10297000122F9C02280A744002296E748002296E6C
:1029800074C002296E28182813281B282927F42828
:10299000332833283B284128472AE727F42AE72809
:1029A00057286028692AE72AE72AE72AE72AE72A38
:1029B000E72AE72AE72AE72AE72AE72AE72AE72A8F
:1029C000E72AE72AE72AE72AE72AE72AE72AE72A7F
:1029D000E72AE72AE72AE72AE72AE72AE72AE72A6F
:1029E000E72AE72AE72AE72AE72AE72AE72AE72A5F
:1029F000E72AE72AE72AE72AE72AE72AE7288528B5
:102A00008D2AE72AE728B328BB28C328CB28D32858
:102A1000E028ED2901290E291B292F293C29492AC3
:102A2000E7295D2966296C2976297B29807876E259
:102A3000B40103A21E22C3227876E2B40B03A21EC5
:102A400022C3227876E2B40D03A21E22C322787636
:102A5000E2B40803A21E22C3227876E2B40903C2BC
:102A60001E22B409FC80F87876E2B40302800920C3
:102A70002006201E03022AE7C21E7876E260F6B422
:102A80000109121BBD121D0F022AE7B40203022A1C
:102A9000E7B40312121D8B400975640EC3122FB1E7
:102AA0008045D21E8041B40802803CB409028037C0
:102AB000B40D05205C31801CB40E08C3740E122FB7
:102AC0004C8011B40F03022AAE24CE50077876E270
:102AD00024AC50137876E2F5F0C2AF7518A07519E2
:102AE0000785F01A1203EED24722104703022E1E6A
:102AF000300903022D9C301501B34003022D9C7850
:102B000077E2B403028006202003201F2FD21F7813
:102B100077E224AC4013E225E0F5F004902CBA9360
:102B2000C5F093C0F0C0E0E2227877E2F5F0C2AFE2
:102B300075189075190885F01A1203EE022E1C12F2
:102B40001B891200AC022E1C740F121CBC022E1C1E
:102B500075640F121BC440E7120100022E1C75643D
:102B60000FD3122FB1022E1C7406126B6F022B2989
:102B7000755D05022B291201A5022E1C30270A744F
:102B800008126BB440031201E2022E1C205C030207
:102B90002B29022E1CD3740F122F4C022B29302705
:102BA000167408126BB4400F7404126BB440081210
:102BB0002F354003022B29022E1C740F122FEA021C
:102BC0002B3F202717121D8B5006120100022E1CCE
:102BD00075640F756D40121D42022B3F75640F1214
:102BE0001D23756D40022B3F740F122E50022E1CB8
:102BF000740F122E91022E1C740F122E78022E1CAE
:102C0000740F122E69022E1C7400126B6F740F1257
:102C10002EAC022B3F7400126BA0740F122EBD025B
:102C20002B3F7400126BB440EC7400126B4F740FA6
:102C3000122EAC022B3F7402126B6F740F122ECE49
:102C4000022B3F7402126BA0740F122EDF022B3F77
:102C50007402126BB440EC7402126B4F740F122E9C
:102C6000CE022B3F7403126B6F740F122EF0022BE7
:102C70003F7403126BA0740F122F01022B3F7403D9
:102C8000126BB440EC7403126B4F740F122EF002EF
:102C90002B3F302703022BDC022E1C2027FA022BAD
:102CA000C57400440F122F9C022B3F7440022CA3CA
:102CB0007480022CA374C0022CA32B4D2B482B50E4
:102CC0002B5E2B292B682B682B702B762B7C2E1CD4
:102CD0002B292E1C2B8C2B952B9E2E1C2E1C2E1C38
:102CE0002E1C2E1C2E1C2E1C2E1C2E1C2E1C2E1C94
:102CF0002E1C2E1C2E1C2E1C2E1C2E1C2E1C2E1C84
:102D00002E1C2E1C2E1C2E1C2E1C2E1C2E1C2E1C73
:102D10002E1C2E1C2E1C2E1C2E1C2E1C2E1C2E1C63
:102D20002E1C2E1C2E1C2E1C2E1C2E1C2E1C2E1C53
:102D30002E1C2BBA2BC22E1C2E1C2BE82BF02BF892
:102D40002C002C082C152C222C362C432C502C64B7
:102D50002C712C7E2E1C2C922C9B2CA12CAB2CB0DD
:102D60002CB57877E2B40103A21F22C3227877E260
:102D7000B40B03A21F22C3227877E2B40D03A21F73
:102D800022C3227877E2B40803A21F22C3227877F5
:102D9000E2B40903C21F22B409FC80F87877E2B4D8
:102DA00003028009202006201F03022E1CC21F7868
:102DB00077E260F6B40109121BBD121D0F022E1C32
:102DC000B40203022E1CB40312121D8B4009756459
:102DD0000FC3122FB18045D21F8041B40802803C3E
:102DE000B409028037B40D05205C31801CB40E0894
:102DF000C3740F122F4C8011B40F03022DE324CEA5
:102E000050077877E224AC50137877E2F5F0C2AF40
:102E10007518A075190885F01A1203EED24722C062
:102E200082C083121DDA121DE612212312212F12F5
:102E3000246C122478D083D082C22020330122C295
:102E400033C2AF7518C0751900751A541203EE22FB
:102E5000543F44C0C2AFF51A751908C245C2442098
:102E60005244121BB7D243803D543F4480C2AFF559
:102E70001A751908D24580E5543F4440C2AFF51A8F
:102E8000751908D244C24520521C121BB7D2438088
:102E900015543F4400C2AFF51A751908D244C24513
:102EA000205203121BA27518C00203EE543F4400C7
:102EB000C2AFF51A75190A7518C00203EE543F44E3
:102EC00080C2AFF51A75190A7518C00203EE543F97
:102ED0004400C2AFF51A75190C7518C00203EE5400
:102EE0003F4440C2AFF51A75190C7518C00203EEC5
:102EF000543F4480C2AFF51A75190C7518C002030F
:102F0000EE543F44C0C2AFF51A75190C7518C002D3
:102F100003EE7405126BA0C22EC22F7401126BA0B7
:102F20007404126BA07406126BA07407126BA07469
:102F300008126BA0227407126BB440067407126B60
:102F40006FC3223027057408126B6F22400C305279
:102F500008C252204403121BB7222052FC122F66D3
:102F6000D252121BA222304414202811543F440094
:102F7000C2AFF51A7519087518C00203EE22C0E039
:102F800024ACD0E0401225E0901FBEF5F00493B4CD
:102F90002008E5F093B42102D322C322A2E69224B2
:102FA000A2E79225C2AFF51A75190D7518C0020374
:102FB000EEC0D0E56D6003022FDB306E05C26E12ED
:102FC00000CED0D0202701B35010202707121D4279
:102FD000121B8922121D23121B8922D0D020270107
:102FE000B340F7756D00121B8922C0E0125F8ED0CE
:102FF000E0543F4400C2AFF51A75190B7518C002B2
:1030000003EEC0F075F0C8D5F0FDD5F0FDD0F0228C
:10301000C0F075F008A2E79282D283123002D28209
:10302000C283123002A2B620B60B005013C3003088
:10303000B612D3800F004008D30020B607C3800427
:1030400000000000B333D5F0CCD0F02212300212D1
:10305000300212300222C283D282D2B6123002D2A1
:103060008312304CC28312304C2275F00778937E65
:10307000007F00E62EFEE6123010F62FFF08D5F096
:10308000F2EED333123010F8EFD333687007789331
:10309000B6FF02C322D322C283D28275F00512008A
:1030A0004730B603D5F0F722223060FC75F00212EB
:1030B0000040D5F0FA12305678937603303C027611
:1030C000052066027601087680087490306617A2A3
:1030D0003E92E5A203B392E4A24192E1A228300914
:1030E00003A204B392E0F608748030660D4557548D
:1030F00087A24092E5A205B392E4F6087480F60830
:10310000F608F612306A403C755B04200A10D20AB9
:10311000C2AF7518C0751900751A031203EE306638
:10312000747899E6789420E34C20E23E20E13278EE
:1031300094E6B6006008B6425C08D268C267E61240
:1031400018438051E55B6016D55B13300A10C20A44
:10315000C2AF7518C0751900751A041203EE02315A
:10316000957894863CD22C02318C863908D23B7AF1
:1031700004798B8009756C28D23A7A05797FE6C488
:10318000540FF709E6540FF70908DAF2D268C2675C
:10319000123097D322123097C32222C32230680EF6
:1031A000C2AF7518B0751900751A001203EE22C26D
:1031B00098C299322009F830992BC29920390E759E
:1031C00031008021D255C2397531008012C0E0C073
:1031D000D0C0F0E581240B40EB75D0101232FCD04A
:1031E000F0D0D0D0E0309805C29830390132C0D04C
:1031F000C0E0C0F075D010E581240B5009D238C270
:1032000039D25502325C303805C238753F00E54688
:1032100024FE4003754602E53F20E71620E61054E1
:1032200007232463C0E074003432C0E0E599220231
:1032300036E1543F232324E2C0E0E43435C0E0E526
:1032400099221567023256023256D567FAB54523E0
:10325000753F0002325C053F2545F545D0F0D0E0D2
:10326000D0D032800E80358038803B803D803F80DA
:103270004B8049B40908754500753F0080D8B421DA
:1032800008754500753F4080CDB44208754500750E
:103290003F8080C2754500753F0080C0B51ED48058
:1032A000B5B51FCF80B0F54080ACF54180A8B545DD
:1032B000C27546401232BE753F0080A080D6854060
:1032C0003312671DD239E533B44603024054B44784
:1032D0000412673322B450108541321266F8C2AC32
:1032E000C239786C7407F22224BF24E64004854179
:1032F0003222C23922C5342534C53422E53124F0C6
:10330000400EE53123241BC0E074003433C0E022BA
:10331000759906C239753100D285228029802E80A8
:1033200030803280338038803F8041804E804C80B6
:103330004A80488043804D804B8049753103F59920
:103340001232F5053122753400740380F1E51E80D8
:10335000EDE51F80E90233D1E53475310F80DF12CE
:10336000041DD246883280D6E53280CFE532600235
:10337000809EA22792E080F2753103A8320532E6E2
:1033800076FF80BAE5321470107408A24492E0A26D
:103390004592E1A22892E280D11470107410A21616
:1033A00092E0A21792E1A21892E280BE14700A7411
:1033B00018A20A92E0D2E180B1147012123EC4C089
:1033C000F0F5F0232345F0D0F0C4D2E3809CE480F4
:1033D00099E533B4410675310402333EB44229E520
:1033E00032600330461DC24653580F53590FC2AFC7
:1033F000E559B55806D2AFD3023403055953590FD6
:10340000D2AFC3744202333BB44404E53380F6B414
:103410004B0280030234F8E53254F8B40832E53246
:10342000540770087419122E50023522B401087422
:1034300019122E69023522B402087419122E78026C
:103440003522B403087419122E910235220233106A
:10345000B42814E532A2E09227756001500375602C
:1034600002756D40023522B4300AE53254F8126B11
:103470006F023522B4380AE53254F8126BA00235D7
:1034800022B48040E5325407FD5403CD65628D625D
:103490007003023522ED7008741A122E5002352284
:1034A000B40108741A122E69023522B40208741A83
:1034B000122E78023522B40308741A122E910235A6
:1034C00022023310B4882EE5325407FD5403CD6533
:1034D000638D637003023522EDA2E09224A2E19293
:1034E000250303441AC2AFF51A75190D7518C012D9
:1034F00003EE023522023310B4430FB53203754F89
:10350000057531077532A802333EB44A1AE53270A8
:10351000E4121BA2C2AF75181075190F751AF012BC
:1035200003EEE53302333BB4450675310602333E04
:10353000B4490FE8C0E0786BE532F2D0E0F87449A6
:1035400080E2B44C0675310E02333EB4460280D49C
:10355000B4470280CFB44F08C22EC22FC23080C4FD
:10356000B45A13E8C0E078B5E2F532D0E0F8745A06
:1035700075310502333E023310023273B462FA022F
:103580003256023256B42A03023256B424EB754046
:1035900032753F43023256F56724C6E56740DA24A8
:1035A000F5E56750D40567023256785AF21567027E
:1035B0003256785BF21567023256785CF215670274
:1035C0003256785DF21567023256785EF215670260
:1035D0003256785FF215670232567860F21567024C
:1035E00032560232940002357C00023582000235E8
:1035F0008500023597000232420002324200023258
:103600004200023242000235AA000235B200023501
:10361000BA000235C2000235CA000235D2000235B6
:10362000DA0002324A0002324A0002324A00023212
:103630004A0002324A0002324A0002324A00023292
:103640004A0002324A0002324A0002324A00023282
:103650004A0002324A0002324A0002324A00023272
:103660004A0002324A0002324A0002324A00023262
:103670004A0002324A0002324A0002324A00023252
:103680004A0002324A0002324A0002324A00023242
:103690004A0002324A0002324A0002324A00023232
:1036A0004A0002324A0002324A0002324A00023222
:1036B0004A0002324A0002324A0002324A00023212
:1036C0004A0002324A0002324A0002324A00023202
:1036D0004A0002324A0002324A0002324A000232F2
:1036E00094B44003023294B44108E599B51E29020E
:1036F0003256B44208E599B51F1E023256B443074C
:10370000E599F540023256B44417E599F541600B4E
:10371000B421005003023256023273753F7E0232EA
:1037200056B47F1AE599B545EF754604753F00120A
:1037300066F8C2ACC239786C7410F202325CC39481
:10374000456009B421004004E59980CCC0E024091B
:10375000F8E599F2D0E005E065417003E280BCE253
:1037600002325685403375320002377AE540448094
:10377000F53375320174017809F212005F12396E67
:103780007400786CF2C23912005FD2851266F8229A
:10379000786CE2B4000122B4070DC082C083123BF2
:1037A000A4D083D08280D9B410D6E540B42846E5B1
:1037B0004124FD50B7C082C0837809E2F58308E256
:1037C000F58208E2B4030A7419123EEB12606E80AF
:1037D0001DB4020A7419123F1A1260338010B4012A
:1037E0000A7419123F23126056800312605AD08364
:1037F000D082023763B42929E54124FE4003023711
:103800006CC082C0837809E2F58308E2F582126019
:1038100072780BF2753203854033D083D082023741
:103820007AB42A0EC082C083125F8ED083D0820207
:103830003763B42B19E54124EF400302376CC08293
:10384000C08312143BD083D08240F0023763B42C83
:103850001EE54124FF400302376CC082C08312146E
:10386000C0D083D08240F0854033F53202377AB43D
:103870002D36E54124FD502DC082C0837809E2F544
:103880008308E2F5821239EF401785832FA88279E9
:103890000B7530011202A6120047D083D082023786
:1038A00063D083D08202376CB42E4BE54124FD50A7
:1038B00042780BE2603DB41D005038C082C083786E
:1038C00009E2F58308E2F5821239EF4022780BE233
:1038D000F53285832FA882790C85323012030B05CF
:1038E0003205320532D083D08285403302377AD018
:1038F00083D08202376CB42F1DC082C083123A2C51
:103900007809E583F208E582F2753202854033D00A
:1039100083D08202377AB43010C082C083123A5FFB
:1039200040CDD083D082023763B4320EC082C083D0
:10393000123BF6D083D082023780B4330EC082C0EF
:103940008312394ED083D08202377A0237807534A1
:10395000007403120225E51E120225E51F1202253E
:10396000743312022574201202251243C222C2852A
:103970007534007423120225E51E120225E51F127C
:103980000225E533120225E532120225E532600EEA
:103990007809E2F5F0E5F012022508D532F4E534B5
:1039A0001202253099FD229033007F28120509DF8D
:1039B000FB22C082C0831239EF402885832FA88262
:1039C00079737530011202E27873E6601CB4FF026D
:1039D00080111685832FA882797375300112026ACF
:1039E000120047D083D082C322D083D082D322E575
:1039F000822418E58334FC5017E5822460F582E5C3
:103A00008334F0F583E58224F8E58334FF500F22F8
:103A1000E5822400F582E5833433F583800CE5826A
:103A20002400F582E5833437F583C322D28575F00F
:103A300001120040D5F0FAE51DB51DFD24219000CE
:103A400000A2B092D5A2D530B001B35003B2D5A335
:103A5000B51DF275F001120040D5F0FA22D322789C
:103A600009E2F58308E2F5822418E58334FC40ED91
:103A7000124389780BE2B4120040E2124397E582C8
:103A800075F006A4F582A8F0E58375F006A428F584
:103A900083E5822400F582E5833450F583C0A2C01B
:103AA00082C08353A2FED083D08243A201758300DB
:103AB00075821E74061269CED0A2752F0078007927
:103AC0006E7530011202E2124397E58224A0F5825E
:103AD000E5833424F58385832FA882790975300125
:103AE00012030B7809E2256EF56E781CE2F9C3E546
:103AF0006E99F56E85832FA882791C7530011202AC
:103B0000A6120047124397E5822460F582E58334CC
:103B10001FF58385832FA882790975300112030B65
:103B20007809E2256EF56E781DE2F9C3E56E99F528
:103B30006E85832FA882791D7530011202A61200AE
:103B400047124397120CE7780C790C7A08E2085474
:103B50000FC4F5F0E208540F45F0F309F5F0E56EF7
:103B6000C395F0F56EDAE685832FA8827914753057
:103B70000812030B7814E56E7A08F9E22908DAFADC
:103B8000F56E85832FA882790C7530081202A61273
:103B90000047752F007800796E75300112026A12A5
:103BA0000047C322126072E532600122C28575347B
:103BB000007403120225E51E120225E51F120225DC
:103BC0007450120225747D1202259000007E7D7FC4
:103BD0000875F000C0F0126072B40203D38001C314
:103BE000D0E033F5F0A3DFEC120225DEE2E534127B
:103BF00002253099FD227809794A75F010E2F30820
:103C000009D5F0F9E56F120C66B3924220260D300B
:103C10004216121D8B401175600480062042097502
:103C20006003A2429227922622302106302F0302FF
:103C30003CD9786474FFF2C231203A0C203B030275
:103C40003E7D120120023CE3120120120E49120DAA
:103C5000886051120B3C70281244E3401DB40A00E6
:103C6000501875F00AA4C0E0124527D0F0B40A003D
:103C7000500825F01252E6023E7D1200CE023E7D33
:103C80002071081257595003023E7D12129F601C8A
:103C900012319DC2AF75182075190F751AEC1203F9
:103CA000EE023CD6123EC45403B40003023D48B4B5
:103CB0000103023D48B40209123ECE123EA2023E6A
:103CC0007D1200B4121681303B0CE5396008120BEE
:103CD000187003023D48123ECED24D1200CEC24DA6
:103CE000023E7DE53960F2B40213788BE675F00A86
:103CF000A4F5F008E625F01252E6023E7D120DEF23
:103D0000601312319DC2AF75182075190F751AEB2B
:103D10001203EE80C1123EC45403B40003023D48B6
:103D2000B40109123ECE123EA2023E7DB40203024D
:103D30003D481200B4121681303AD8120120120EFA
:103D400049120A736002808E755300754F05C230A8
:103D5000C22FC22EC082C0831213DED083D0825005
:103D600006123EA2023E7DE58224CEE58334FF505A
:103D700008123EBB4003023E32E53720E006302702
:103D800009305406123EA2023DD3E538600DC082D0
:103D9000C083120C37D083D08250E92045E6121D33
:103DA000C240E1786374FFF2123F8140D71239B20A
:103DB00040D2C204C241A268924CD24B121BA21242
:103DC000319DC2AF75181085831985821A1203EED2
:103DD0001200AC123EBB5008E53720E603023E7DE0
:103DE000D203C23EC205D240D202C23F7557001272
:103DF00030A9C082C083121681D083D082120BF208
:103E0000203A05203B1580751212E8500712129FC8
:103E100060208015120A736019800E1212E84009A2
:103E2000E5396005120B186009D24D1200CEC24D63
:103E3000804B202705121D8B40EF786474FFF2B28F
:103E400027756D40D24A12319D755E03121B89D2CF
:103E500005C240302710C2AF75187085831985825E
:103E60001A1203EE800EC2AF751860858319858221
:103E70001A1203EE1200AC122F17122F437864E2CD
:103E8000B4020A741C123F1A126033800BB401088A
:103E9000741C123F23126056786474FFF2C23BC256
:103EA0003A22D24D12319DC2AF75182085831985F3
:103EB000821A1203EE120100C24D22E582249CE513
:103EC0008334FF22E4A22492E0A22592E1227553DA
:103ED0003CD54F16C2AF751830751900854F1A12B0
:103EE00003EE754F05D22F7552FF2230592B543FE8
:103EF00044C0C082C083C0E0C2AF7518E08583199A
:103F000085821A1203EED0E0C2AFF51A75190E754C
:103F100018C01203EED083D082223059FC543F44A3
:103F20008080CF3059F3543F444080C63059EA5422
:103F30003F440080BD7863E2B40118C082C083783A
:103F400062E2F5827861E2F583741C123F2312600D
:103F5000568019B4021AC082C0837862E2F5827872
:103F600061E2F583741C123F1A126033D083D08251
:103F7000786374FFF2227862E582F27861E583F279
:103F800022123FCA4025126072B4000520682880C2
:103F900022B4011920682030592EC2AF7518C0759F
:103FA0001900751A091203EE205A1DD322B402FB20
:103FB0002068E4740180027402C0E0123F767863E6
:103FC000205B027864D0E0F2C322786BE2B4010592
:103FD00020680FD322B4020530680780F6B40302CC
:103FE00080F1C322C203C23EC204C241C2857534FD
:103FF000007405120225E51E120225E51F12022596
:104000002212005F123FE4E533120225E53412026A
:10401000253099FD229000007B307C001203B9C04E
:10402000E0123FE4E533120225D0E0120225E53428
:104030001202253099FD2212005F123FE4E533128F
:1040400002257973E712022509DDF9E5341202250C
:104050003099FD22122F12755314D209C206C28E56
:10406000C28CC2ADC2ABC2ACC2AF7581B590407854
:10407000C082C08375D00032D2AFD28CC207D203C7
:10408000C23ED204C241D205C240755700C2667515
:1040900057001230A9C26775570012319BD203C274
:1040A0003ED204C241C205C240120047D203C23E02
:1040B000D204C241C205C2401266F8C2ACD2991203
:1040C000400175A61E75A6E112053E755314D298DF
:1040D000D285D203C23ED204C24112020CB40AF00D
:1040E000F53412020CB51EF512020CB51FEF1202C8
:1040F0000CF533B46D0302412BB46E03024146B498
:104100006F03024175B470030241D2B471030242DD
:1041100000B46603024211B465030243BFB46303F3
:10412000024233B4690302429680A5AF3412020CF6
:104130006F709D124001D28575F01E120040D5F0BF
:10414000FAC2AF02000012020CFD1424E040231258
:10415000020CFC12020CFEAF3412020C6F70138EB4
:10416000F08C2FA8F079738D301202E2124037756F
:1041700053140240D012020CFD1454E070F41202E9
:104180000CFC12020CFEEDFA787312020CF608DA3F
:10419000F9AF3412020C6F70D9C203C23EC204C21E
:1041A000418EF07873ED126A3DC0A2C082C0835385
:1041B000A2FE8C8385F08243A2017583007582C1C3
:1041C000ED1269CED083D082D0A212400175531473
:1041D00080A0AF3412020C6F7098C01EC01F126A0C
:1041E000D6D01FD01E120A5412053F1205321205F6
:1041F0003D1239A71240047553140240D002417297
:10420000AF3412020C6F70F5124015755314024052
:10421000D0AF3412020C6F600302417212005F12C1
:10422000005F123FE4E5331202251243C20240D080
:1042300002417212153840F812020CF58312020C7A
:10424000F58212020C70E912020C70E4AF34120213
:104250000C6F70DCC01EC01F85831E85821F120A72
:1042600054752F00780079737530011202E278736B
:10427000E6C3951EC3951FD01FD01E251E251FF611
:10428000752F007800797375300112026A120047A9
:104290001240010240D0AF3412020C6F7092126AC9
:1042A00098600574010242BC126AB3600574020290
:1042B00042BC1242F312432612054EE4C0E0123F04
:1042C000E4E533120225D0E0C0E0120225E5341205
:1042D000022575F003120040D5F0FA123FE4E533F1
:1042E000120225D0E0120225E5341202253099FD94
:1042F0000240D0900000C082C08379737420126A9B
:1043000050D083D08285832FA88279737530201294
:10431000026A120047E5822420F58250020583E5F7
:1043200083643070D122903000C082C0837973746E
:1043300020126A50D083D082C082C083E5822400DC
:10434000F582E5833420F58378737420126A3DC0CA
:10435000A2C082C083C082C08353A2FED083D08219
:1043600043A2017583007582C174201269CED08387
:10437000D082D0A2D083D082E5822420F582500260
:104380000583E583644870A122C0E078B3E583F239
:1043900008E582F2D0E022C0E078B3E2F58308E2DB
:1043A000F582D0E0227400120225740012022574F6
:1043B0000012022574001202257400120225220246
:1043C000417274651202257447120225740B1202A1
:1043D000257405120225740412022574C0120225E8
:1043E0007430120225740012022574001202257422
:1043F00000120225740312022574E81202257400CB
:104400001202257400120225740012022574001293
:104410000225744112022574011202257400120251
:104420002574001202257400120225740012022560
:104430007400120225740012022574001202257401
:104440000012022574001202257400120225740065
:104450001202257400120225740012022574001243
:104460000225E5341202253099FD2245EB467E46B1
:10447000B146E445D345D345D345D345D347174744
:104480004A478F47A047B147C247D345D345D34595
:10449000D347E447F545D3488A48064816482B4891
:1044A00050486D49724D4C48C44D024D2745D34587
:1044B000D349C049D149E249F0499748A74BE64C56
:1044C000744BC14C0B4C994C2E4C514CBC4CDF4D99
:1044D000CB48E149FE4AAC4B014B2045D345D3457F
:1044E000D348FE7F008FF0C0F0120B3CD0F0AFF04D
:1044F00070330FEF24F0402D8FF0C0F0121674D0FF
:10450000F0AFF0202C1F303A0E12012075F050123F
:104510000040D5F0FA80CEEFB40A01E4C0E012000A
:10452000B4D0E0C322D322C082C0833009037553C4
:10453000F012167D303A0D1201201244E35012742D
:10454000FF024551202C07740F30090580E3120447
:1045500034D083D08222125D051200AC7553F0D2A4
:1045600009C228C24BD24AC229C22AC22BD24AC28D
:1045700006C203C23ED204C241C205C240D202C238
:104580003FC22C124527B40A0040030245D375F000
:104590000AA4C0E0C203D23ED204C241C205D24046
:1045A000124527B40A0040030245D3D0F025F0FF9E
:1045B000602624D8FE24C4401A90446BEE25E00403
:1045C00093C0E0EE25E093C0E0EF22125CD212002F
:1045D000AC809E1200CE8099124527B40B02800257
:1045E00080F11200AC125CD20268B312153840E3BD
:1045F0001200B4124527B40A0040030245D3243008
:10460000FD124527B40A0040030245D32430F51FAC
:104610008D1E120A5480B41200B4124527B40A0049
:10462000400302463D6003B40113C0E0124E87D040
:10463000F0400AB454005005AFF0FEC322D322B4B8
:1046400001028013B40302800EB405028009B4068F
:10465000028004C322D322F5F0786EE265F060F5A3
:10466000786FE265F060EE7870E265F060E778768A
:10467000E265F060E07877E265F060D980D51246B7
:104680001750030245D3EE122F7E40F7786EE2C03A
:10469000E07400F2EE12463FD0E0786EF240E4EEB5
:1046A000F2EFC20C6002D20C12077E1205850245A1
:1046B000CB12461750030245D3EE122F7E40F778F7
:1046C0006FE2C0E07400F2EE12463FD0E0786FF285
:1046D00040E4EEF2EFC20D6002D20D12077E120529
:1046E000850245CB12461750030245D3EE122F7EAA
:1046F00040F77870E2C0E07400F2EE12463FD0E07E
:104700007870F240E4EEF2EFC20E6002D20E1207B1
:104710007E1205850245CB12461750030245D3EEA3
:10472000122F7E40F77876E2C0E07400F2EE124677
:104730003FD0E07876F240E4EEF2EFC2146002D2AD
:104740001412077E1205850245CB1246175003024C
:1047500045D3EE122F7E40F77877E2C0E07400F286
:10476000EE12463FD0E07877F240E4EEF2EFC21569
:104770006002D21512077E1205850245CB1200B4E5
:10478000124E874008C0E012624ED0E022D32212BF
:10479000477D40097878F21208A20245CB0245D342
:1047A00012477D40097879F21208A20245CB0245F2
:1047B000D312477D4009787AF21208A20245CB0253
:1047C00045D312477D4009787BF21208A20245CBFF
:1047D0000245D312477D4009787CF21208A20245B7
:1047E000CB0245D312477D4009787DF21208A20220
:1047F00045CB0245D312477D4009787EF21208A2CC
:104800000245CB0245D31200B4124E874012F53553
:104810001207400245CB1200B4124E8740027003CB
:104820000245D3F53612075F0245CB1200B412459C
:1048300027B40A0040030245D3FD54FC700FEDA2DB
:10484000E09224A2E192251207010245CB0245D352
:104850001200B4124527B40A00400302486AC31389
:10486000700892211206000245CB0245D31200B413
:10487000124527B40A004003024887C31370089208
:10488000221206000245CB0245D31200B41245277E
:10489000B40A0040030248A4C3137008925D1206D4
:1048A000000245CB0245D31200B4124527B40A00DA
:1048B00040030248C1C3137008925B120600024510
:1048C000CB0245D31200B4124527B40A00400302BC
:1048D00048DEC313700892081206000245CB024559
:1048E000D31200B4124527B40A0040030248FBC3A8
:1048F00013700892541206000245CB0245D31200F1
:10490000B4124527B40A004003024918C3137008C3
:1049100092711206000245CB0245D31200B4124533
:1049200027B40A00400302496CC313703F9260121F
:104930004527B40A00400302496CC313702E9261EC
:10494000124527B40A00400302496CC313701D408E
:104950001B925E124527B40A00400302496CC31340
:10496000700A4008925F1206000245CB12068A02C6
:1049700045D31200B4124527B40A004003024994FB
:10498000B40300500FA2E19250A2E0B3924F12067E
:10499000000245CB0245D31200B4124527B40A00E9
:1049A00040030249BDB403005013C259C25A600704
:1049B000D259B40202D25A1206000245CB0245D3A4
:1049C0001200B47537FE124FB140030245CB0245C9
:1049D000D31200B47537FE12504C40030245CB028F
:1049E00045D31200B4124F9C40030245CB0245D37D
:1049F0001200B412502F40030245CB0245D31200DF
:104A0000B4124527B40A004003024AFE75F00AA416
:104A1000C0E0124527B40A0040030245D3D0F02578
:104A2000F0B42000502B7873F6124527B40A0040EA
:104A3000030245D375F00AA4C0E0124527B40A006A
:104A400040030245D3D0F025F0787AF61257D340D0
:104A500003024AA9124527B40A004003024AA9C327
:104A60001370EEB3337879F6121681303A3B1201A7
:104A7000207873E6C0E07879E6C0E0787AE6C0E0B6
:104A8000120D88601E1256B54019125E02787876B3
:104A9000FFD0E0787AF6D0E07879F6D0E0125716B9
:104AA0000245CBD0E0D0E0D0E00245D31200B412F2
:104AB000167D303A121201201256B55041125D4F48
:104AC000EF1257160245CB302C34120434B40A06C8
:104AD0001257350245CBB40A00502375F00AA4C022
:104AE000E0124527B40A004003024AFED0F025F048
:104AF000B420005009125D4F1257160245CB0245F3
:104B0000D31200B4124527B40A004003024B3FB44D
:104B10000600502B75F033A4F57212098F0245CBB5
:104B20001200B4124527B40A004003024B3FB406FA
:104B300000500C75F033A4F57112098F0245CB02B9
:104B400045D31200B4124527B40A004003024B5F5C
:104B5000C3C0D0801BB40A3674FFD0D0024B8CB4D3
:104B60000A2ED3C0D0124527B40A004003024B5589
:104B700075F00AA4FA124527B40A004003024B8ECE
:104B80002AD0D092E7F5F0B480028004C322D0D0BE
:104B9000D322124E874028C0E01218DED0E0401F1A
:104BA000C0E01200B4124527B40A004003024BBD16
:104BB000B402005008A2E0926FD0E0C322D0E0D34C
:104BC00022124B42401DF5F0700575F0FF8006B4CF
:104BD000FF030245D374002400F8E5F0F21209D176
:104BE0000245CB0245D3124B42401DF5F0700575CE
:104BF000F0FF8006B4FF030245D374022400F8E5F9
:104C0000F0F21209D10245CB0245D3124B42401BB0
:104C1000F5F070030245D3B4FF030245D3740124B9
:104C200000F8E5F0F21209D10245CB0245D3124B50
:104C300042401BF5F070030245D3B4FF030245D395
:104C400074052400F8E5F0F21209D10245CB0245C3
:104C5000D3124B42401BF5F070030245D3B4FF035F
:104C60000245D374062400F8E5F0F21209D102459A
:104C7000CB0245D3124B42401DF5F0700575F0FF95
:104C80008006B4FF030245D374032400F8E5F0F274
:104C90001209D10245CB0245D3124B42401BF5F01D
:104CA00070030245D3B4FF030245D374042400F813
:104CB000E5F0F21209D10245CB0245D3124B424036
:104CC0001BF5F070030245D3B4FF030245D374070C
:104CD0002400F8E5F0F21209D10245CB0245D312C7
:104CE0004B42401BF5F070030245D3B4FF0375F04F
:104CF0000074082400F8E5F0F21209D10245CB0255
:104D000045D3124B92401DA26F92627873F6752FB5
:104D10002A78C4797375300112026A1200471206AC
:104D2000000245CB0245D3124B92401DA26F926305
:104D30007873F6752F2A78C5797375300112026A77
:104D40001200471206000245CB0245D31200B412EE
:104D50004527B40A004003024D9275F00AA4C0E052
:104D6000124527B40A004003024D8FD0F025F0C051
:104D7000E0124527B40A004003024D8D6003B401E0
:104D80000CA2E0D0E01251D640050245CBD0E002A3
:104D900045D3B40AFA124527B40A004003024D8FE6
:104DA0006016B401EA752F2A782779FF753008124A
:104DB00003A01200470245CB752F2A78277900758A
:104DC00030081203A01200470245CB1200B4124E65
:104DD0003B4043E583703C75F008C0F0124527B4B2
:104DE0000A004003024E116003B40125A2E0E5373A
:104DF00013F537D0F0D5F0E2743C124E257877E504
:104E000082C4540FF608E582540FF61212F60245DA
:104E1000CBD0F00245D3B40AFA753700124E2512F2
:104E200012F60245CB75F00A7873F608D5F0FB222E
:104E3000124E3BE58245837001D322124527B40A06
:104E4000004003024E8575F00AA4F582C082124527
:104E500027B40A004003024E83D082258275F00AEF
:104E6000A4F58285F083C082C083124527B40A006E
:104E70004003024E83D083D0822582F58250020502
:104E800083C32274FFD322124527B40A00400302D1
:104E90004EA975F00AA4C0E0124527B40A004003E9
:104EA000024EA9D0F025F0C322D322010000000059
:104EB00000000000000A00000000000000000004E4
:104EC000060000000000000000080E0300000000C3
:104ED00000000000010702000000000000000A06B8
:104EE00008010000000000000402040F00000000A0
:104EF00000000806090809000000000000010E0576
:104F00000F0500000000000A0C0A090B0300000056
:104F100000040E0B00040502000000080E0607083E
:104F200004070100000001050A040D080E75F00ACF
:104F3000797F770009D5F0FA78A4EA603F24F2502F
:104F400007EA24F328F87A0DE6540FF66029EA14EC
:104F500075F00AA424ABF5827400344EF583798889
:104F60007E007B0AE493F5F0E6A42E2775F010840A
:104F7000FEA7F0A319DBED08DACEC322D322124537
:104F800027B40A004003024F9AB40800500C24A032
:104F9000F5827400340FF583C322D32212168130B8
:104FA0003A6E125E02120B80C322124F7E40618065
:104FB0000D9000007537FE8008124E3040521200EE
:104FC000B412167D303A1A120132C037120BF2D0E9
:104FD00037125E02125E224037753800125BEFC353
:104FE00022302C2C120434C0E024F6D0E040217A88
:104FF0000D78A4F608EAC0E0E8C0E0124527B40A3C
:10500000004003025012D0F0A8F0D0F0AAF0DAE38A
:10501000D322D0F0A8F0D0F0AAF0B40BF3C3740EF2
:105020009AFAC082C083124F2DD083D082809B1207
:105030001681303BDBE53924FD24FC40D3125E0AA7
:10504000120B91C322124F7E40C6800A900000804E
:1050500008124E3040BA1200B4121681303BB1C073
:1050600037120BF2D037125E0AE539600B24FD24AB
:10507000FC409D125E8E4098753800125BEFC32293
:10508000124E30400B125D4F753700125BEFC3229A
:10509000D322124F7E400B125D4F753700125BEF2B
:1050A000C322D322124E30402F120BF212519940DC
:1050B00027C082C0831200B4124527B40A004003FF
:1050C0000250D8D083D082600FB40900500AF5F0A6
:1050D000D3E433D5F0FCC322D3221250A4400DC038
:1050E000E0120BA2D0E04237120BCDC3221250A423
:1050F000400EC0E0120BA2D0E0F45237120BCDC329
:1051000022124527B40A004003025188607AB4098C
:10511000005075F5F0D3E433D5F0FCF4FF752F247F
:1051200078A179737530071202E2787375F007E69B
:105130005FF608D5F0F9752F2478A17973753007DB
:1051400012026A1200479024A885832FA8827973DF
:105150007530081202E2787375F008E65FF608D53C
:10516000F0F985832FA882797375300812026A12CC
:105170000047E5822408F58250020583E582247801
:10518000E58334D750C3C322D322124E30400812D5
:105190000BF2125199B322D3227873E6080808085B
:1051A0000856B4FF02D322C322125222402475F0C3
:1051B00008842427F582E4342AF58385832FA88286
:1051C00079617530011202E2E56105F013D5F0FC5A
:1051D000E4227401D322C0D0125222404175F0085B
:1051E000842427F582E4342AF58305F0747F23D5DF
:1051F000F0FCC0E085832FA882796175300112022E
:10520000E2D0E05261D0D05003F4426185832FA8F0
:1052100082796175300112026A120047C322D0D030
:10522000D322B42800501224F6500EC0E09052C889
:10523000936004D0E0C322D0E0D322C0641200B453
:10524000121681203A13203B42C23AC23BD064D3AB
:105250002212129F70F30252C0120132120D887096
:10526000F0123EC45403B400030252C0B40103025E
:1052700052C0B4020280D21200B4121681303BC96F
:10528000120132120B1870C10252C0120132E539FC
:1052900060B7120DEF70B2123EC45403B4000302A3
:1052A00052C0B4010280A2B402030252C01200B480
:1052B000121681303A93120132120A736002808909
:1052C000C23AC23BD064C3220101010101010101C4
:1052D00001000101010100000000000000010101C6
:1052E000010100000001D203C23EC204D241C20546
:1052F000D240D202C23F207140B4012B12523B4037
:1053000038E583458270321200B4121681203B0BBF
:10531000303A26120B5E7027024556E539601A12A4
:105320000B6F701B024556C0E01251A97009D0E006
:10533000C0E04010025350D0E01200CE22D0E01264
:105340003ECE80F512523B40F4E53720E50280ED79
:105350001200B4D0E0B40A25124527B40161124509
:1053600027B4005B125D5EC2AF7518C075190A7470
:105370000A543F4440F51A1203EE025539B40B1E8D
:10538000753700124FB94037C2AF7518C075190A8A
:10539000740B543F4440F51A1203EE025539B40C15
:1053A000217537001250514016C2AF7518C07519DB
:1053B0000A740C543F4440F51A1203EE02553902A8
:1053C0005535B40D1B12508040F5C2AF7518C0752D
:1053D000190A740D543F4440F51A1203EE02553970
:1053E000B40E1BC2AF7518C075190A740E543F4431
:1053F00040F51A1203EE12518A40C4025539B40F17
:105400002E7537009000641259BD401BC2AF75184D
:10541000C075190A740F543F4440F51A1203EE1276
:105420005CD21200B480DA7003025539025535B4EB
:10543000101B1250DA4088C2AF7518C075190A7473
:1054400010543F4440F51A1203EE025539B4111BB3
:105450001250ED40D7C2AF7518C075190A741154B7
:105460003F4440F51A1203EE025539B4121B125193
:105470000140B9C2AF7518C075190A7412543F447F
:1054800040F51A1203EE025539B41425124527B41B
:10549000029A124527B40094125DD0C2AF7518C0AD
:1054A00075190A7414543F4440F51A1203EE02555C
:1054B00039B4151E753700124FAA4079C2AF75185E
:1054C000C075190A7415543F4440F51A1203EE02D0
:1054D0005539B4161E7537001250454058C2AF7585
:1054E00018C075190A7416543F4440F51A1203EE99
:1054F000025539B4171B125092403AC2AF7518C00A
:1055000075190A7417543F4440F51A1203EE0255F8
:1055100039B41F030255D5B420030255EDB421035D
:10552000025580B4220302565CB4230302568BB4A6
:1055300027030256411200CE22125CD21200AC2286
:105540007400126B6FC2AF7518C075190AE5645408
:105550003F4400F51A1203EE80E27400126BA0C201
:10556000AF7518C075190AE564543F4480F51A12E6
:1055700003EE80C87400126BB440DF80C375641BF7
:10558000124527B4000280D2B4010280B3B40202F3
:1055900080E280A17402126B6FC2AF7518C07519DA
:1055A0000CE564543F4400F51A1203EE808E740239
:1055B000126BA0C2AF7518C075190CE564543F4456
:1055C00040F51A1203EE02553C7402126BB440DE31
:1055D00080C275641B124527B4000280D1B4010259
:1055E00080B2B4020280E202553575641B12452771
:1055F000B400028028B401028008B402028039029B
:1056000055357403126B6FC2AF7518C075190CE570
:1056100064543F4480F51A1203EE02553C740312A1
:105620006BA0C2AF7518C075190CE564543F44C037
:10563000F51A1203EE02553C7403126BB440DE807F
:10564000C17404126B6FC2AF7518C075190B741B4F
:10565000543F4440F51A1203EE02553C124527B45C
:105660000008741B122E5002553CB40107741B1223
:105670002E9180F3B40207741B122E7880E9B403D4
:1056800007741B122E6980DF025535124527C0E0D2
:1056900024FBD0E0401CA2E09224A2E19225030367
:1056A000441BC2AFF51A75190D7518C01203EE022E
:1056B000553C0255359028A07F2085832FA88279FC
:1056C000737530081202E2120A736010E582240832
:1056D000F582E5833400F583DFE0C322787AE6B40F
:1056E000FF0280F6C0E07879E6A2E0B3926FC3745F
:1056F000209FFFD0E0900FE9D32275F008A424A0EA
:10570000F582E5F03428F58385832FA882797375B7
:1057100030081202E22275F008A424A0F582E5F018
:105720003428F58385832FA8827973753008120297
:105730006A120047229028A07F2085832FA88279B3
:10574000FF7530081203A0120047E5822408F58295
:10575000E5833400F583DFE2221256B5400822D0FB
:10576000E01200CED322C0E0D203C23EC205D24036
:10577000C202D23F7557001230A9306F0C12523B53
:1057800040DDE53720E70280D6D0E025E0F5F004E3
:1057900090579F93C0E0E5F093C0E0E5F0032257F7
:1057A0006157F0576158115761583558565871581C
:1057B000A158A958B158B958C158CA58D358DC583B
:1057C000E558EE576158F75922592B59345761590A
:1057D0003D595EB41A00501225E0C0E090579F93E7
:1057E000B45709D0E0A393B46104C322D0E0D3221C
:1057F0007537009000641259BA4037C2AF7518C0AF
:1058000075190A7401543F44C0F51A1203EE025987
:105810008E7537009000011259BA4016C2AF751844
:10582000C075190A7403543F44C0F51A1203EE02FE
:10583000598E0257617537009000321259BA4045AF
:10584000C2AF7518C075190A7405543F44C0F51AE3
:105850001203EE02598E125996402AC2AF7518C033
:1058600075190A7406543F44C0F51A1203EE025922
:105870008E1200B4121681303A0B1201201256B566
:105880005006B40703025761125D5EC2AF7518C0BF
:1058900075190A7407543F44C0F51A1203EE0259F1
:1058A0008E741D122E50025991741D122E910259A0
:1058B00091741D122E78025991741D122E6902598D
:1058C0009175641D12559402599475641D1255AE5C
:1058D00002599475641D1255C902599475641D12BC
:1058E000554002599475641D12555A0259947564B5
:1058F0001D1255740259947537009000641259BAFC
:105900004018C2AF7518C075190A7413543F44C0CB
:10591000F51A1203EE125CD280DD70030259910277
:10592000576175641D12560202599475641D125612
:105930001D02599475641D1256380259947537002A
:10594000900FA01259BA402AC2AF7518C075190A33
:105950007418543F44C0F51A1203EE02598E120017
:10596000B4121681303A0B1201201256B55006B40B
:105970001903025761125DD0C2AF7518C075190ABC
:105980007419543F44C0F51A1203EE02598E125C8A
:10599000D21200ACD3221200B4121681303A19127E
:1059A0000120120D887011E5824583600B125D4F56
:1059B000753700125BEFC322D3221200B4C0371236
:1059C0005A01702B121681303A2B120120C082C06E
:1059D000831256B5D083D0824015125D4F125E02FD
:1059E000125E22400AD037753800125BEFC322D016
:1059F00037D3740122303B04E53970F3D037D3E458
:105A000022E5822460E58334F05003025A75E58272
:105A100075F008A4F51BC0F0E58375F008A4D0F07C
:105A200025F0F51CE51B2420F51BE51C3400F51CB6
:105A3000851C2FA81B79737530061202E27906784F
:105A400073B6FF0508D9FAE422E51B2408F51B50BC
:105A500002051CA3E582B4E807E583B403028012C3
:105A6000E583700CE582B464028007B432028002E0
:105A700080BE740122120D6379067873B6FF0508A3
:105A8000D9FAE422A3E582B4A8EBE583B40FE6805B
:105A9000E1D203C23EC204D241D205C240D202C208
:105AA0003F751E30751F30121538D267D266125DF1
:105AB0004F121681203B12303AD7120120125E029B
:105AC000025B001200CE0268B3125B1940F512159A
:105AD00038402D1200AC12167D302CE7120434B47D
:105AE0000B03025B00B40A0050D92430F51E1216D5
:105AF0007D302CCF120434B40A0050C72430F51F77
:105B00001200AC9000007538007537FE125BEF1282
:105B10000B80120B91120A5422203A2C303B29E5BB
:105B200039600624FD24FC401F125E0A1200B412E4
:105B3000167D203A0B302C10120434B40B0A800668
:105B4000120120125E02C322D322C203D23EC2043B
:105B5000D241D205C240D202C23FD267C2661216FB
:105B600081203A03303BE3125D4F125E0290000049
:105B70007537FF125BEF120B80120B911215384034
:105B80001D1200B4125BBD402C2430C0E01200B4E2
:105B9000125BBDD0F0401E85F01E2430F51F120AA6
:105BA000541200ACD203C23ED204C241D205C2405C
:105BB000D202C23F22751E30751F3080E175F00B96
:105BC000C0F0121681203A0DD0F075F00BC0F01223
:105BD0001681303A0A120120D0F0D5F0F0D322D04D
:105BE000F0C3740B95F060F5B40A027400C322C0D0
:105BF00082C083E5822460F582E58334F0F583502A
:105C000008125C6ED083D08222D083D082C082C042
:105C100083125C51D083D082120BCDC082C083121C
:105C20000CE785832FA882797375300812026A12F7
:105C30000047D083D08222E5822460F582E5833458
:105C40001FF58385832FA88279387530011202E20F
:105C500022E5822460F582E583341FF58385832F56
:105C6000A882793875300112026A12004722C08278
:105C7000C083E5822460F582E5833431F583858332
:105C80002FA882793875300112026A120047D0833A
:105C9000D082C082C083E5822480F582E5833431DE
:105CA000F58385832FA882793775300112026A1235
:105CB0000047D083D082C082C083120D1F85832FFE
:105CC000A882797375300812026A120047D083D017
:105CD00082229000007B307C001203B9C0E0752F57
:105CE00000780079737530011202E27873E6D0F023
:105CF000C395F0F6752F00780079737530011202A4
:105D00006A1200472278737628087664752F3278F5
:105D100010797375300212026A12004722752F3211
:105D2000781079737530021202E27873B62817087A
:105D3000B66413C2AF7518C075190A7401543F4494
:105D400040F51A1203EE787376FF0876FF80BD7572
:105D50003800787375F00876FF08D5F0FA229000C5
:105D60002885832FA88279FF7530181203A01200AE
:105D7000479000407FF985832FA88279FF753020F6
:105D80001203A0120047E5822420F5825002058309
:105D9000DFE4752F2478A079377530011202E29084
:105DA00024A07F2085832FA88279FF7530201203DD
:105DB000A0120047E5822420F58250020583DFE42B
:105DC000752F2478A0793775300112026A120047C6
:105DD0009031207F0885832FA88279FF75300812C3
:105DE00003A0120047E5822408F58250020583DFF4
:105DF000E4752F31788079FF7530081203A0120006
:105E00004722787F79737A058006788B79787A03D0
:105E1000E608540FC4F5F0E608540F45F0F709DA28
:105E2000EF22C082C083900000120D06125F5B70EB
:105E30001AE5828583F0D083D082B5824FC5F0B554
:105E4000834AC082C083F58385F082A3E583B403CF
:105E5000D8E582B4E8D3900FA0120D3E125F5B70BC
:105E60001AE5828583F0D083D082B5821FC5F0B554
:105E7000831AC082C083F58385F082A3E583B40FC3
:105E8000D8E582B4A8D3D083D082C322D322C082E3
:105E9000C083900000120D06125EFA701AE582852A
:105EA00083F0D083D082B5824FC5F0B5834AC082DB
:105EB000C083F58385F082A3E583B403D8E582B47B
:105EC000E8D3900FA0120D3E125EFA701AE582859B
:105ED00083F0D083D082B5821FC5F0B5831AC0820B
:105EE000C083F58385F082A3E583B40FD8E582B43F
:105EF000A8D3D083D082C322D322EFC0E0C23278AD
:105F00008479787A06EA30E004E6088002E6C45430
:105F10000FFFEA30E004E7098002E7C4540FB40F32
:105F200010BF0F10EA6406600B20321ED0E0FFE4C1
:105F300022BF0F06D0E0FF7401222032F7F5F08F68
:105F40003E6F6002D232DABD80DFE5F0C3953E508D
:105F500002F4041460D6B408DB80D1787F79737AB8
:105F6000057401B6FF02800FB7FF02800AE6677072
:105F7000060809DAF8E422740122905F82C082C028
:105F800083327581B575D000125CD20268B3C082CD
:105F9000C08390014175F0FAE4F0A3D5F0FB9002C4
:105FA0003B75F002E4F0A3D5F0FBD083D08222E56C
:105FB000822418E58334FC4033E582540375F003F2
:105FC000600F75F00C14600975F03014600375F003
:105FD000C0E5830303F583E58203034583758301ED
:105FE0002441F58250020583E5F0C322E582246056
:105FF000F582E58334F0F5835037E58224F8E583B4
:1060000034FF402DE582540375F003600F75F00CEA
:1060100014600975F03014600375F0C0758302E5F3
:106020008254FC0303243BF58250020583E5F0C350
:1060300022D32274AAC082C083C0E0125FAFD0F026
:10604000400FC5F055F0F8E5F0F4F5F0E055F048F4
:10605000F0D083D08222745580DBE5825583B4FF73
:1060600004125F8E227419123F2C740080C774FFD3
:1060700080C3C082C083125FAF401BF5F0E0C5F063
:1060800020E00A0303C5F00303C5F080F3E5F054F4
:1060900003D083D082227400D083D0822230591959
:1060A00012024E7869E2F5F07877E6B5F0028009E1
:1060B0007869F220560420573E2279657876E67595
:1060C000F00A84C445F0F5F0E3B5F028097877E6E6
:1060D00075F00A84C445F0F5F0E3B5F017125F8E51
:1060E000C2AF7518C075190B741A543F4400F51AE5
:1060F0001203EE223057C279677876E675F00A848B
:10610000C445F0F5F0E3B5F027097877E675F00AB5
:1061100084C445F0F5F0E3B5F016125F8EC2AF759A
:1061200018C075190B741A543F4400F51A1203EE87
:1061300022601AB4071BF5F0A22992E0A22B92E18B
:10614000A22A92E255F0C36001D3920722A227B39C
:106150002240E3B40903A24B22B40A0C88F0C0F039
:10616000121D62D0F0A8F022B40B03A24D22B40E8F
:1061700003A24C22B40F07C3E55D6001D322B41221
:1061800006A2457244B322B41305A244822822B465
:106190001405A244B02822B41503A24522B4190A5A
:1061A000C3202705E55E6001D322B41A0AC3302755
:1061B00005E55E6001D322B440067400126BB42280
:1061C000B441067401126BB422B442067402126B1D
:1061D000B422B443067403126BB422B444067404AC
:1061E000126BB422B445067405126BB422B4460691
:1061F0007406126BB422B447067407126BB422B44F
:1062000048067408126BB422B45006A2247225B357
:1062100022B45105A224B02522B45205A225B024EF
:1062200022B45305A224822522B46105A228824CFF
:1062300022B46205A228B04C22B46402C322A22870
:1062400022FFCE3C0600000000FF010F0008C0E066
:10625000249CD0E0401C75F00884C0E005F07480F8
:1062600023D5F0FCF5F0D0E09062419355F0600248
:10627000C322D3227878E2126131B392B47879E202
:10628000126131B39294787AE2126131B39295201F
:106290005D15206012787BE2126131B39283787CC5
:1062A000E2126131B3928222C0E0123056789374C8
:1062B00005C44407F608D0E0C0E023A2E392E5A2BB
:1062C000E292E3542AD2E7F608D0E0C0E0A2E392DB
:1062D000E1A2E492E3542AD2E7F608D0E0A2E692E3
:1062E000E1A2E792E3540AD2E7F6748008F608F6D2
:1062F00008F675F00778937E007F00E62EFEE61222
:106300003010F62FFF08D5F0F2EED333123010F82C
:10631000EFD33368700B7893B6FF06123097C380C3
:1063200004123097D32222305DFC304AF9C24AE48D
:10633000C0E0787DE2126131D0E092E0C0E0787E8A
:10634000E2126131D0E092E1A22892E2A229722AFF
:10635000722B92E3A227B392E4C0E07406126BB4EE
:10636000D0E092E5C0E07407126BB4D0E092E6C0D2
:10637000E07408126BB4D0E092E71262A874035084
:1063800004126417221263F9C082C0837894E6C0B5
:10639000E054071263A3D0E0C454071263CED08345
:1063A000D08222A21E301401B3400F30E01B30E136
:1063B0001CD31227B5C31227B52220E00C30E20D02
:1063C000C31227B5D31227B522B31227B522A21FB5
:1063D000301501B3400F30E01B30E11CD3122AEA24
:1063E000C3122AEA2220E00C30E20DC3122AEAD3BB
:1063F000122AEA22B3122AEA22E55AB402052275C9
:106400005A022250FA755A02C2AF7518C0751900A7
:10641000751A351203EE22E55A6019D5E014C2AFA1
:106420007518C0751900751A3F1203EE7406126BC9
:106430006FE4F55A2275D90075D800E572F4F5FDC0
:1064400075DD4275DE00D29743B74075D840D2AEB5
:1064500022C0D0C0E0E5D830E40975DE00126478CF
:1064600075DE4D75D840D0E0D0D032741525EEF5EC
:10647000EE740235FEF5FE22B200E571B44C004028
:106480002CB47F004061B4B200403FB4E50050DB63
:1064900020000D74D625EEF5EE740035FEF5FE22D3
:1064A000745425EEF5EE740335FEF5FE2220000D42
:1064B000742B25EEF5EE740035FEF5FE2274FF25F3
:1064C000EEF5EE740335FEF5FE2220000D746B250B
:1064D000EEF5EE740035FEF5FE2274BF25EEF5EE06
:1064E000740335FEF5FE2220000D744B25EEF5EE0B
:1064F000740035FEF5FE2274DF25EEF5EE740335EB
:10650000FEF5FE22C0F0C0E0C0D0745875F000D592
:10651000F0FD20B339D5E0F4C2AFD294D295D28346
:10652000D282D205C240D202C23FC203C23ED204CE
:10653000C24175F032120040D5F0FAD203C23EC219
:1065400004C24175F032120040D5F0FA80DCD0D0A0
:10655000D0E0D0F0C28B32C28C758AA6758CAED2D8
:106560008CC0D0C0E0200904E554600675A61E75F5
:10657000A6E1E57060021570B249304905B24830B5
:106580004805D0E0D0D032C0F075D008E5812407AE
:106590005004D2558045051D12668012044CE51D3D
:1065A00020E03820E13512666C200936204105A232
:1065B00028B39204E51D541F701B1266AAD24A121A
:1065C0006BCBE4B55524B55040B5524BB55D53B5D2
:1065D0005E59B5535A12663D126274D0F0D0E0D0C5
:1065E000D032E51D541F60EA80F1D555D9C24B2049
:1065F00052D42044D1305005121D62400AC228C234
:106600004BD24AD243D24A80BDD550BDC24B7552FF
:10661000FFD230D23380B2D552B2C22EC22FC23096
:1066200080AAD206D55DA8C20680A4155E80A3D537
:1066300053A3754F05300903025F7A808FE4B55488
:106640000AB5510BB5460CB56D1022155480F215E4
:106650005180F1D546F1D23880EDD56DEDD26E8006
:10666000E9C285203902D2851266F832E51DA2E220
:10667000303E0292033041029204304002920522E1
:10668000A2029291A2039290A2049292A2059293E6
:1066900020060C30080320070675DE00D29722E59D
:1066A00071B41900400375DE4D2230510A202707CE
:1066B000C229C22AC22B220556E556540704F5F01A
:1066C000740103D5F0FCC0E0C22A302E0AD0E0C02D
:1066D000E054F86002D22AC229302F0AD0E0C0E08C
:1066E00054806002D229C22B30300AD0E0C0E0547E
:1066F000A06002D22BD0E02275C800C2ADC2AC753A
:10670000CBFF75CA9875CDFF75CC98759853C29814
:10671000C299D2ACC2BC75C8347599062275C8003E
:10672000C2ACC2AD75980075CC2B75CDEBD2AD75F2
:10673000C8042275C800C2ACC2AD759800E58A24B1
:106740002BF5CC540F658C24EBF5CDD2AD75C80478
:106750002274FFF580F590F5A0D209C206755500A8
:10676000C228C24BD24AD296E4F53875F010784A66
:10677000F208D5F0FBC244C245C224C225C216C2EB
:1067800017C218C219C21AC21BC21CC21DC22CC217
:106790002EC22FC230755201755300C233D238C297
:1067A00039755B01755C01C20AC20B751E30751F1D
:1067B00030754610E4F53FF540E541F531F533F528
:1067C00035F536786EF2786FF27870F27871F2788B
:1067D00072F27872F27874F27875F27876F27877ED
:1067E000F274637878F2787DF274047879F2787EC6
:1067F000F27400787AF27400787BF27400787CF29C
:10680000E4F550F556F558F559F53BF560F55D1290
:106810006B19753AFF753CFF751D047437F547F524
:1068200048F549F54AF54BF54CF54DF54ED2207536
:106830004F0575510178A87A0576FF08DAFBC24644
:10684000D247C24BC24CC24DC252C251C2537562F2
:10685000FF7563FF120230786B7400F2C26E756DC3
:1068600000D27078B5E4F2756F02C207C2067554A3
:10687000FA75A61E75A6E112103B75A61E75A6E157
:10688000758901758A9F758CAEC2B9D2A9D28CD296
:10689000851266F8D2BA43B704C28AD2AA12643506
:1068A000D2AFC282D2B6C255125F8E2230600312BE
:1068B000309722C2AF12053E020000780175F0FF4A
:1068C00074FFF608D5F0FBF890000074FFF0A3E524
:1068D000822400E58334FD50F2E4C2F0900000020F
:1068E00068F2C2AF758E11758F0175A70575D0005E
:1068F00080C97581B578FF763E1216221267511253
:10690000014D120EE41268AC12053F125D1DC2AFBC
:10691000751880751905751A0B1203EEC209C26845
:10692000D266C269D267120113C209205550E581AF
:10693000B4B54678FFB63E3DC241D205C240121BF7
:106940008912609DC268D266C269D267D2431216AC
:1069500081203B1C203A193053CF755D0512319DC3
:10696000C2AF7518C0751900751A071203EE80B909
:10697000123C2980B4D285763ED2857581B5D28508
:10698000C255C2AF7518C0751900751A581203EEBA
:1069900075F0FA120040D5F0FA0268B38AF0C0F040
:1069A0008CF0C0F08EF0C0F043A22012FFF053A292
:1069B000DFD0F0AEF0D0F0ACF0D0F0AAF022A2AF71
:1069C000C0D0C2AF790212699CD0D092AF228EF0B3
:1069D000C0F0FE53A2FEE5832490F583500302002D
:1069E00000A2AFC0D0C2AFE582F45480C39582FA52
:1069F000C39E5037F404FE43A201C082C08353A259
:106A0000FEC082C083EA790912699C53A2FED0833A
:106A1000D082E5822AF5825002058343A201D08309
:106A2000D082E5822AF5825002058353A2FE7909BD
:106A3000EE12699CD0D092AFD0F0AEF022C082C0EE
:106A4000839000C1F9E6F008A3D9FAD083D082225E
:106A5000F8E5832490F5835003020000E493F7A344
:106A600009D8F922F8E5832490F583500302000049
:106A7000E493F3A309D8F922F8E5832490F5835031
:106A8000030200007900E49329F9A3D8F9C0E0E5F6
:106A9000832470F583D0E022900000E4F5F0C0F08C
:106AA000E4126A78D0F025F0C0E0E583643070F03D
:106AB000D0E022903000E4F5F0C0F0E4126A78D023
:106AC000F025F0C0E0E583644870F0D0E02290004B
:106AD000C1F0A3D9FC22798074FF126ACE53A2FEC2
:106AE000900000C0A2C082C083C082C08353A2FEB7
:106AF000D083D08243A2017583007582C174801255
:106B000069CED083D082D0A2E5822480F582500263
:106B10000583E583644870CB22789B75F009E4F621
:106B200008D5F0FB780075F00974FFF208D5F0FB8A
:106B300078017483F278047483F278057483F278B0
:106B4000067483F27807743CF278087400F222B479
:106B50000900501088F0C0F0249BF876FFD0F0A810
:106B6000F0D3D24A22C0E0126BB4D0E0B35031B4BB
:106B70000900502B88F0C0F0F5F02400F8E2C5F0D1
:106B8000C0E0249BF8E6600CD0E0B402028007B4B9
:106B900003068002D0E0A6F0D0F0A8F0D24AD322BB
:106BA000B40900500D88F0C0F0249BF87600D0F0B6
:106BB000A8F0C322B40900501088F0C0F0249BF85C
:106BC000E6D0F0A8F06002D322C322C24ED55F0502
:106BD000D24E755F3C789B75F009E66003B4FF0503
:106BE00008D5F0F62220E708D5E002800CF680F008
:106BF000304EED14F6B480E8E4D24AF6E8B4A205CB
:106C000075600580DBB4A3D875600680D33099FD2C
:106C1000C299F59922540FB40A005003243022245B
:106C20003722126C15126C0D22C0E0C4126C1512C2
:106C30006C0DD0E0126C15126C0D22740D126C0DDF
:106C4000740A126C0D227428126C0DE583126C29E3
:106C5000E582126C297429126C0D221266F8C2ACFE
:106C6000C28522C0D03099FDD2851266F8D0D022DC
:106C7000C0E0126C3B7445126C0D7472126C0D7492
:106C800072126C0D742D126C0DD0E0126C0D74200C
:106C9000126C0D126C467420126C3B22740D1202A1
:106CA00025740A120225740A120225740A1202259A
:106CB000740A120225740A120225740A120225743B
:106CC0000A1202253099FD2275F06484C0F0243048
:106CD000120225D0E075F00A84C0F024301202259B
:106CE000D0E0243012022522000000000000000045
:106CF0000000000000000000000000000000000094
:106D00000000000000000000000000000000000083
:106D10000000000000000000000000000000000073
:106D20000000000000000000000000000000000063
:106F9000000000000000003C434647544147533E78
:106FA0003C5645523D47313231363E3C46495849C0
:106FB000443D20203E3C4E414D453D505233313101
:106FC0005345762E312E31312E313231363E3C440E
:106FD0004154413D30382D30362D31302030303A5B
:106FE0003331203E3C2F434647544147533E00280F
:106FF0004729284255462E434647290000533D3C29
:00000001FF
